:106770000000090200000301FA0400FA0500030A00
:106780000A5A0B001E0C00FA0D00030E00040F0144
:1067900064100096120132130AFA14010217010A5A
:1067A0001801FA1905321A010A1B01FA1C05321FD9
:1067B000FFFF20FFFF23011E2400642A00FA2B00A4
:1067C000FA2C50782D003D2E00463000643250786F
:1067D0003300003432FA3501643601643701503831
:1067E0000A643C00643E003C3F000140FFFF41144E
:1067F00050420A5A430AC84405324500B44600FADA
:106800004C00FA500C0C510596520A32530B465468
:106810000A96570546590A465A32FA5B010A5C0A3B
:10682000325E000A5F00FE64021167FFFF6A0A3CE5
:106830006B00006C329673000174000178013279AC
:1068400001327E006481006484FFFF8A00019D0A9A
:10685000969E00019FFFFFA0FFFFA2000AA3FFFF7B
:10686000A4FFFFA5FFFFA6FFFFA7FFFFA8FFFFA94B
:10687000FFFF0101241500002F003C4701244802BE
:10688000025601024EFFFF58000261FFFF66000141
:106890008500AF8600018700FA890107990000A1F1
:1068A00000FAFAFAFA0101241500002F1E3C4701F4
:1068B000244802025601024EFFFF58000261FFFF0A
:1068C0006600028500AF8600018700FA89010799FA
:1068D0000000A10000FAFAFA0101241500002F1EA1
:1068E0003C4701244802025601014EFFFF580000B8
:1068F00061FFFF66000085FFFF86FFFF87FFFF89BE
:106900000102990000A10000FAFAFA0065006F0088
:10691000790083008D009700A100AC00B600C00094
:10692000CA00D400DE00E800F200580060006800F1
:10693000700078008000880090009800A000A800F7
:10694000B000B800C100C800D000D800DF00E600E9
:10695000EE00F600410047004D00530059005F0073
:1069600065006C00710077007D00830089008F0056
:1069700095009B00A200A700AC00B200B900C000C7
:0F698000C500CA00D200D500DD00E100E700EF3E
:1033100090089EE090012AF090089FE0900099F0BC
:103320009008A0E09000B9F09008A1E09000E2F0D1
:103330009008A2E090008EF09008A3E09000D4F0F6
:103340009008A4E09000F2F09008A5E09000C6F08C
:103350009008A6E09000E4F09008A7E0900114F037
:103360009008A8E0900178F09008A9E0900179F029
:103370009008AAE090017AF0900178E0700C90013A
:1033800079E0700690017AE060028004C221800238
:10339000D2217433900163F07436900164F0742D7F
:1033A000900165F07431900166F07420900167F02F
:1033B0007431900168F07432900169F074439001A7
:1033C0006AF0747990016BF0746C90016CF0742069
:1033D00090016DF0742090016EF0742090016FF0F8
:1033E0007420900170F07420900171F02290089682
:1033F000E0FEA3E0FF7402D39F74019E400C90672F
:1034000070120048E493F599804C900067E0D394E3
:10341000054014900896E0FEA3E0FF90677012004C
:1034200048E493F599802F900067E0D3940440140A
:10343000900896E0FEA3E0FF9067A3120048E49393
:10344000F5998012900896E0FEA3E0FF9067D612EF
:103450000048E493F599900896126AAF900896E0B8
:10346000FEA3E0FFEFB43507EEB40103754C002274
:1034700075A71085F97285FA737E017F00E57312D6
:103480006AA1E5722FFF50010E8E598F5A900025C8
:10349000E0FCA3E0FDEF2DFDEE3CFC8C5B8D5C229F
:1034A000E55CF5FBE55BF5FCD29322E55CF5E9E52F
:1034B0005BF5EAD29422E55CF5EBE55BF5ECD291A5
:1034C00022E55CF5EDE55BF5EED29222E55CF5FDDB
:1034D000E55BF5FED28722E55CF5CEE55BF5CFD264
:1034E0009022AE59AF5A740A8E048F05FF126A916A
:1034F0008C5B8D5CAE59AF5A740A8E048F05FF1237
:103500006ABC8C598D5AE55A45596013740AC395A3
:103510005AFFE49559FE8E598F5A785B126AF4E58A
:1035200072A85BB80015D3955C4010E572C3955C3A
:10353000FFE4955BFE8E5B8F5C8010E5722424C3F4
:10354000955CFFE4955BFE8E5B8F5CAE5BAF5C745D
:10355000246F4E700B755C23755B007572018003E0
:10356000757200229000A0E0B40104C2068002D26D
:10357000069000A1E0B40104C2078002D2079000C7
:10358000DEE075F0DCA4FFAEF0740A8E048F05FF58
:10359000126A9190088EECF0A3EDF074078C068D02
:1035A00007126AA174038E048F05FF126A919000BE
:1035B00021ECF0A3EDF07E017F0090009CE0126A08
:1035C000A19000DFE08E048F05FF126A91740AFF5C
:1035D000126A918D5F9000E8E075F0DCA4FFAEF018
:1035E000740A8E048F05FF126A91900892ECF0A382
:1035F000EDF09000EAE060139000EAE0F5F0741658
:1036000084FF7E00EF9008BAF0800674649008BAD8
:10361000F09000E0E090007EF090012EE0FE90003F
:10362000DCE08E0088F0A4FFAEF0EF9008C2F090CE
:10363000012AE090089EF09000E2E09008A1F0904E
:10364000008EE09008A2F09000D4E09008A3F090E3
:103650000114E09008A7F0900178E09008A8F0909D
:103660000179E09008A9F090017AE09008AAF0A210
:1036700021B34016900178E0700C900179E070065B
:1036800090017AE060028002C221900178E0B430BB
:103690000F900179E0B4470890017AE0643B600242
:1036A0008004D2228002C22274E390007DF0900058
:1036B000C9E0B40B0874E390007DF0805A9000C913
:1036C000E0B419129000DFE09068F612008CE493E9
:1036D00090007DF080419000C9E0B41E129000DFA0
:1036E000E090691412008CE49390007DF0802890A3
:1036F00000C9E0B428129000DFE090693E12008C0F
:10370000E49390007DF0800F9000C9E0B4460890EB
:1037100000C0E090007DF0900081E0FE9000C6E0E7
:10372000B5063F900083E0FE9000E4E0B5063390DC
:103730000082E0FE9000F2E0B50627900084E0FEF3
:10374000900099E0B5061B900085E0FE9000FFE038
:10375000B5060F900086E0FE900100E06E70030257
:10376000391D7407900115F0900099E0B4010674BA
:1037700000900099F0900099E0B402067400900067
:10378000E4F0900099E0B4030674009000F1F0902A
:1037900000F2E0B4012774009000AEF0741C9001B8
:1037A00018F074009006EAF074009006EBF09000B8
:1037B000C6E0B4020674019000C6F080339000C6E3
:1037C000E0B4021A741C9000AEF07400900118F07E
:1037D00074009006EAF074009006EBF0801274001A
:1037E000900118F074009000AEF0741C9006EAF09E
:1037F0009000E4E0D39401402674009000ADF07492
:103800001B900117F074009006E6F074009006E734
:10381000F09000C6E0600674009000C6F080329020
:1038200000C6E0601A741B9000ADF07400900117A0
:10383000F074009006E6F074009006E7F0801274D1
:10384000009000ADF07400900117F0741B9006E634
:10385000F09000B9E06014740990011CF0740090BD
:1038600006DAF074009006DBF0800C740090011C06
:10387000F074099006DAF09000FFE060147407908D
:103880000119F074009006DEF074009006DFF080FD
:103890000C7400900119F074079006DEF09001009E
:1038A000E06014740890011AF074009006E2F0745D
:1038B000009006E3F0800C740090011AF0740890F8
:1038C00006E2F0D2209000C6E0900081F09000F275
:1038D000E0900082F09000E4E0900083F090009986
:1038E000E0900084F09000FFE0900085F0900100EF
:1038F000E0900086F0900099E090089FF09000B969
:10390000E09008A0F09000F2E09008A4F09000C6CB
:10391000E09008A5F09000E4E09008A6F090008701
:10392000E0FE9000B9E06E60449000B9E06014746D
:103930000990011CF074009006DAF074009006DB28
:10394000F0800C740090011CF074099006DAF0907D
:103950000087E060069000B9E07002D2209000B9C4
:10396000E0900087F09000B9E09008A0F09000FC93
:10397000E0B40117900031740FF0A374FFF09000D1
:1039800033E4F0A3F074029000FCF09000FCE0B48B
:103990000341900033E0FEA3E0FF900031E0FCA380
:1039A000E0FD126AEC7410126AA17408120039EF7B
:1039B00090007AF0EF700674FF90007AF074009037
:1039C00000FCF0900032E090007BF0900031E0903D
:1039D000007CF090008DE090008AF090008CE090E8
:1039E0000089F09000BBE0C3941E50569000BBE0ED
:1039F000F404241E90008BF090008BE075F00A8494
:103A0000FF7E008F7290008BE075F00A84ADF07C31
:103A1000008D73900089E0D39573400D900089E08C
:103A2000C39573900089F0800F900089E0240AC349
:103A30009573900089F0057290008AE025729000DD
:103A40008AF090008AE090004DF090004DE0D39411
:103A500024400B90004DE0C3942490004DF0900062
:103A60004DE0240690004EF090004DE0240C9000B4
:103A70004FF090004DE02412900050F090004DE087
:103A80002418900051F090004DE0241E900052F058
:103A900090004EE0D39424400B90004EE0C3942459
:103AA00090004EF090004FE0D39424400B90004FD4
:103AB000E0C3942490004FF0900050E0D394244051
:103AC0000B900050E0C39424900050F0900051E01F
:103AD000D39424400B900051E0C39424900051F003
:103AE000900052E0D39424400B900052E0C3942401
:103AF000900052F0900059E4F090004DE0B4240C96
:103B00009000597401F090004D7401F090005AE457
:103B1000F090004EE0B4240C90005A7401F0900034
:103B20004E7401F090005BE4F090004FE0B4240C80
:103B300090005B7401F090004F7401F090005CE421
:103B4000F0900050E0B4240C90005C7401F0900000
:103B5000507401F090005DE4F0900051E0B4240C4A
:103B600090005D7401F09000517401F090005EE4EB
:103B7000F0900052E0B4240C90005E7401F09000CC
:103B8000527401F090008DE0FE9000F0E02E900065
:103B900060F0900060E064126007900060E0B42480
:103BA00006900060E004F0900060E0D39424400BA5
:103BB000900060E0C39424900060F0900060E0D337
:103BC0009412400D900060E0C39412900061F08068
:103BD0000A900060E02412900061F075501290008D
:103BE000D3E0900053F0900053E075F00684AFF0FE
:103BF0007E00EF4E7006900053E004F0900053E01A
:103C0000B425069000537401F0900053E024069010
:103C10000054F0900053E0240C900055F0900053B5
:103C2000E02412900056F0900053E02418900057C2
:103C3000F0900053E0241E900058F0900054E0D320
:103C40009424400B900054E0C39424900054F090CE
:103C50000055E0D39424400B900055E0C394249089
:103C60000055F0900056E0D39424400B900056E0AD
:103C7000C39424900056F0900057E0D39424400B56
:103C8000900057E0C39424900057F0900058E0D380
:103C90009424400B900058E0C39424900058F022E4
:103CA000C293C294C291C292C287C290E5B554EF4A
:103CB000F5B5E5B554DFF5B5C296C295C2A0C29779
:103CC000C2A2C2A1E5B554BFF5B5E5B5547FF5B5BF
:103CD000E5B554FBF5B5C208755D469000D6E070B9
:103CE00005756C028003756C037554007553009064
:103CF000001874FFF0A374DCF0C20EC210C212C22E
:103D000014C216C21874C8900035F074C8900039F7
:103D1000F074C890003DF074C8900041F074C890F1
:103D20000045F074C8900049F0755200755100C20A
:103D300003754500E56EB40903756E007562009069
:103D40000027E4F0A3F0756F10C20BC20CC20DC2C5
:103D50000275560075550090001AE4F0A3F090002B
:103D60001CE4F0A3F0C22575580075570090009828
:103D7000E075F032A4FFAEF090002FEEF0A3EFF06C
:103D8000900088E4F022755A00755900AE59AF5A78
:103D90007402C39F74019E5003023E4490677012E8
:103DA0000048E49390008C126AD20FBF00010EE02D
:103DB000FC906770120048ECFEE493FFEEC39F5046
:103DC00026AE59AF5A0FBF00010E9067701200481F
:103DD000AE59AF5AE493FC906770120048E4939098
:103DE000008C126AD2ECF0AE59AF5A906770120094
:103DF00048E49390008C126AD2E0FC906772120043
:103E000048ECFCE493FDECD39D40199067721200DE
:103E100048E493FC906770120048E49390008C1281
:103E20006AD2ECF0AE59AF5A74022FFF50010E8ED9
:103E3000598F5A785A740126F6500418E436F64021
:103E400003023D8C22755A00755900AE59AF5A7461
:103E500033BE00039F5003023F1290687212004865
:103E6000E49390008C126AD20FBF00010EE0FC9028
:103E70006872120048ECFEE493FFEEC39F5026AE3A
:103E800059AF5A0FBF00010E906872120048AE5928
:103E9000AF5AE493FC906872120048E49390008C4F
:103EA000126AD2ECF0AE59AF5A906872120048E430
:103EB0009390008C126AD2E0FC906874120048EC77
:103EC000FCE493FDECD39D4019906874120048E423
:103ED00093FC906872120048E49390008C126AD2AE
:103EE000ECF0AE59AF5A742D6F4E7006755A33759B
:103EF0005900AE59AF5A74022FFF50010E8E598FE0
:103F00005A785A740126F6500418E436F640030233
:103F10003E4B22755A00755900AE59AF5A7433BEE4
:103F200000039F5003023FE09068A5120048E4930D
:103F300090008C126AD20FBF00010EE0FC9068A5C1
:103F4000120048ECFEE493FFEEC39F5026AE59AF3B
:103F50005A0FBF00010E9068A5120048AE59AF5A23
:103F6000E493FC9068A5120048E49390008C126AD8
:103F7000D2ECF0AE59AF5A9068A5120048E4939085
:103F8000008C126AD2E0FC9068A7120048ECFCE4B6
:103F900093FDECD39D40199068A7120048E493FC70
:103FA0009068A5120048E49390008C126AD2ECF05D
:103FB000AE59AF5A742D6F4E7006755A337559004D
:103FC000AE59AF5A74022FFF50010E8E598F5A7896
:103FD0005A740126F6500418E436F64003023F19DD
:103FE00022755A00755900AE59AF5A7433BE00039A
:103FF0009F50030240AE9068D8120048E4939000AE
:104000008C126AD20FBF00010EE0FC9068D812003B
:1040100048ECFEE493FFEEC39F5026AE59AF5A0F13
:10402000BF00010E9068D8120048AE59AF5AE49311
:10403000FC9068D8120048E49390008C126AD2EC8D
:10404000F0AE59AF5A9068D8120048E49390008CB3
:10405000126AD2E0FC9068DA120048ECFCE493FDAE
:10406000ECD39D40199068DA120048E493FC906804
:10407000D8120048E49390008C126AD2ECF0AE594A
:10408000AF5A742D6F4E7006755A33755900AE597C
:10409000AF5A74022FFF50010E8E598F5A785A74FE
:1040A0000126F6500418E436F64003023FE722E505
:1040B0000C906348F828287302414CA22EB34008A4
:1040C000E5B54408F5B58006E5B554F7F5B5807C4F
:1040D000A22EB34008E5B54402F5B58006E5B55417
:1040E000FDF5B58067A22EB34008E5B54404F5B5EB
:1040F0008006E5B554FBF5B58052A22EB34008E525
:10410000B54410F5B58006E5B554EFF5B5803DA290
:104110002EB34008E5B54420F5B58006E5B554DF7B
:10412000F5B58028A22EB34008E5B54440F5B5802A
:1041300006E5B554BFF5B58013A22EB34008E5B52A
:0C4140004480F5B58006E5B5547FF5B568
:106348000240B80240BB0240D00240E50240FA02D7
:08635800410F0241240241390A
:10414C002275A71085F97285FA737E017F00E573DD
:10415C00126AA1E5722FFF50010E8E598F5AAC5B7B
:10416C00AD5CEF2DFDEE3CFC8C5B8D5CD293D29460
:10417C00D291D292D287D290E55CF5FBE55BF5FC4F
:10418C00E55CF5E9E55BF5EAE55CF5EBE55BF5ECA3
:10419C00E55CF5EDE55BF5EEE55CF5FDE55BF5FE67
:1041AC00E55CF5CEE55BF5CF75A7002285F9728548
:1041BC00FA737E017F00E573126AA1E5722FFF503E
:1041CC00010E8E598F5A7E017F76900111E0126A92
:1041DC00A1AC59AD5AED2FFFEC3EFE8E5B8F5CE52A
:1041EC005CF5E9E55BF5EA90007EE4F07412900072
:1041FC0063F02285F97285FA737E017F00E57312F4
:10420C006AA1E5722FFF50010E8E598F5A90088EBD
:10421C00E0FCA3E0FDEF2DFDEE3CFC8C5B8D5CE542
:10422C005CF5FBE55BF5FC22056322A2D8B3400CE0
:10423C00C296C295C2A0C297C2A2C2A1A2D9B340D3
:10424C00089000E0E090007EF075D8402285A771C0
:10425C0075A710A2D8B34002C293A2D9B34002C230
:10426C0094A2DAB34002C291A2DBB34002C292A282
:10427C00DCB34002C287A2DDB34002C29075D840C5
:10428C008571A72290F800E4936406600280FE75A5
:10429C00B50075840175A70075FF8075EF06900059
:1042AC005FE4F075C91075A70F75A1C775A70075E8
:1042BC00D90075CE0C75A70F75F1FE75F2FF75F36D
:1042CC000775F47875A4BA75A5FF75A60775AE00C9
:1042DC0075AFFF75D48175D5FF75D6FF75D7FF7592
:1042EC00A70075A20175A14775F80975D80075D995
:1042FC000475DA0975DB0975D84075A71075D800F7
:10430C0075D90475DA0975DB0975DC0975DD097574
:10431C00DE0975DF0975D84075A70075E60875E7E5
:10432C001075BC0175BE0475BD6C75BE0775BDA05E
:10433C0075BE0875BD0175BC0075BB1875BC2075C4
:10434C00BA0875E88075D11375A70F75E10575E28C
:10435C000075C740123CA0759700759780740A12BF
:10436C006A817597C0E5975420700280F8758F02AA
:10437C0075A700D2AF75980075A90C75A70F75AB12
:10438C004375ADFB75AC1E75A71075C91875CA00C1
:10439C0075CB0075C80475A700758912758E0475E8
:1043AC008C00758A00C2A9D28C758D00758B00D2D9
:1043BC00ABD28E75B62075D944C299C22474C8F597
:1043CC00097508001200F875A70FE5FB90006DF059
:1043DC00E5FA90006EF0E5F990006FF075A700908B
:1043EC00F800E493F52612021790089FE0D394038B
:1043FC00500790089FE0B40106740090089FF07479
:10440C00019000D5F090089FE0906360F828287325
:10441C00802A802875A70F75F30F75A700A2A340FB
:10442C000674029000D5F0801375A70F75F31775FD
:0C443C00A700A2A4400674029000D5F076
:0C63600002441C02441E0244200244358A
:104448009000D5E0B4022AC2231205B67402900087
:10445800D5F090089FE090636CF82828738010804E
:0F4468000E74009000E4F0800674009000F1F0F4
:0C636C0002446502446702446902447167
:104477008028D2231204D574019000D5F090089FAC
:10448700E0906378F82828738010800E74009000FD
:0A449700E4F0800674009000F1F0DC
:0C63780002448F02449102449302449BB3
:1044A1001233109000DFE07006740A9000DFF09084
:1044B10000C0E0700674E39000C0F09000C6E00414
:1044C100900081F09000B9E004900087F01235640B
:1044D10090F807E493900074F0900074E0440A901F
:1044E1000074F0900074E054FE900074F074069033
:1044F1000065F07401900066F090F802E49390007A
:1045010067F07403900068F07405900069F0743AE4
:1045110090006AF0740690006BF0900067E0B404BC
:1045210006740490006BF0900067E0B40506740512
:1045310090006BF0740690006CF090F804E4939096
:104541000070F07400900071F090F805E493900011
:1045510072F090F806E493900073F074FF90007588
:10456100F0123D86900067E0B40505123F138011FB
:10457100900067E0D394054005123E458003123F49
:10458100E19000FBE090007AF09000B2E090007BB7
:10459100F09000B3E090007CF0A2B6B39204A2B315
:1045A100B39205A2A4B3921EA2A3B3921F90007668
:1045B100E4F0756E00743A90078CF074FD90078DED
:1045C100F0900077E4F0756D01900063E4F09000E5
:1045D100D6E0B40106741A900063F0C21D75620042
:1045E100C209D20AC202757000C22012009E755E15
:1045F10000756A0075600075643275650075660046
:10460100756700756800756900900027E4F0A3F0F4
:10461100756B00D2B2D2A4D2B0D2B1D2A3D2A7D2FA
:10462100A6D2A5D2B7900098E0D394FA400674FAC6
:10463100900098F07E017F0090007CE0126AA190CA
:10464100007BE02FFF50010E900031EEF0A3EFF060
:10465100EFD394FFEE940F4007900031E4F0A3F004
:1046610090007AE0700674FF90007AF09000D6E036
:104671007005756C028003756C039000D7E0D394CC
:1046810001400674009000D7F09000DDE0C3940A69
:104691005006740A9000DDF09000E7E070067401A6
:1046A1009000E7F09000E7E0B4FF0674FE9000E7A9
:1046B100F09000EEE0D394FE400674FE9000EEF020
:1046C100900114E0D3940240067401900114F0901B
:1046D100012AE0D394014006740190012AF074018B
:1046E1009000F4F074019000F5F074009000FCF07B
:1046F10074299006D2F0742A9006D6F0D29C9000CC
:10470100C7E0D39404400674049000C7F09000F908
:10471100E0D39404400674049000F9F0E56FD3945B
:10472100104003756F109006D3E0D3940C400674CB
:10473100009006D3F09006D7E0D3940C40067400A5
:104741009006D7F09006DBE0D3940C4006740090FD
:1047510006DBF09006DFE0D3940C4006740090066F
:10476100DFF09006E3E0D3940C400674009006E37A
:10477100F09006E7E0D3940C400674009006E7F051
:104781009006EBE0D3940C400674009006EBF0D257
:10479100EC75CF01A298B34005C298120697E54C7B
:1047A1006006A299B3B340028005C299120B78E565
:1047B1004D64016005E54DB4040280D5C28E7E10C2
:1047C1007F00E563126AA1E58D75F010A4FDACF0E0
:1047D100EF2DFDEE3CFCE58B75F01084FF7E00EDC6
:1047E1002FFFEC3EFE8E538F54D28E9000B9E060C5
:1047F100099000B9E0C3943D40028056900029120F
:104801006AAF900029E0FEA3E0FF90002BE0FCA33B
:10481100E0FDEFB5053CEEB50438B21AA203B34092
:1048210013A21AB34008E5B54404F5B58006E5B511
:1048310054FBF5B590002BE0FEA3E0FF90002DE0C6
:10484100FCA3E0FDEF2DFDEE3CFC90002BECF0A372
:10485100EDF09000C6E060099000C6E0C39403400B
:10486100030248EA122745A203B35009900076E0FB
:10487100C3941F400280069000B0E0F544E5447502
:10488100F002A4FFAEF0900894EEF0A3EFF09000D8
:104891009DE0C395604007E55EC3955F50079008B2
:1048A10094E4F0A3F0AE2DAF2E900894E0FCA3E0C9
:1048B100FDEFD39DEE9C4015E5B554BFF5B59000D5
:1048C100C6E0B40206E5B54480F5B5801C900076DB
:1048D100E0C3942E5013E5B54440F5B59000C6E011
:1048E100B40206E5B5547FF5B59000C6E0B40324E3
:1048F100122860AE2DAF2E900894E0FCA3E0FDEFEE
:10490100D39DEE9C4008E5B54440F5B58006E5B57C
:1049110054BFF5B5A2B6300401B35003024F29A22A
:10492100B6300401B35003024F29A2B6300601B3D9
:104931005003024DE1756D009000B9E0B43D13A242
:1049410006B34008E5B554FBF5B58006E5B544046A
:10495100F5B5055DA208B3B35013AE53AF54900043
:1049610018E0FCA3E0FDEDC39FEC9E4003024A89E1
:10497100E56CB4032EA225B34022E55DB424037592
:104981006C01E55DC3942450069000637401F0E569
:104991005DD3942440067402900063F0755D01D2EA
:1049A100258062E56CB40206756C01755D24E55DD8
:1049B100B42405755D01804D900063E07038E55DBC
:1049C100C3942450069000637401F0E55DD39424F0
:1049D10040067402900063F0E55DC394245002D256
:1049E1001DE55DD394244002D21DC296C295C2A09A
:1049F100C297C2A2C2A19000D6E0B40105123CA0A8
:104A01008003755D01AE55AF56AC53AD54EF2DFD2E
:104A1100EE3CFC7403FF126A918C558D569000B9DF
:104A2100E060099000B9E0C3943D400280439000EA
:104A310029E0FEA3E0FF9000B9E08E048F05FF128C
:104A41006A9174018C068D0712003990002DEEF0E9
:104A5100A3EFF090002DE0F8A3E090002BC8F0A3A5
:104A6100C8F0900029E4F0A3F0C21AE5B554FBF5B3
:104A7100B5A2A4B34002C21EA2A3B34002C21FA2A8
:104A81001DB34002C21D803AAE55AF56AC53AD5472
:104A9100EF2DFDEE3CFC74018C068D071200398E62
:104AA100558F56E56CC39402500DAC53AD5474B69A
:104AB100C39D740E9C40028009123CA074069000B4
:104AC10063F0E55DB424127403900063F0D21D908D
:104AD10000D6E0B40103123CA0AE57AF58AC53ADC1
:104AE10054EF2DFDEE3CFC8C578D58AE53AF54EF77
:104AF100D39DEE9C401190001FE0FAA3E0FBEBC3B5
:104B010094E8EA94034002800690001F126AAF9075
:104B1100001CE0FEA3E0FFAC53AD54EF2DFDEE3CD5
:104B2100FC90001CECF0A3EDF09000D6E0B4011D68
:104B3100AE53AF547405126AA174038E048F05FF3E
:104B4100126A91900018ECF0A3EDF08016AE53AF0D
:104B5100547403126AA17401120039900018EEF026
:104B6100A3EFF0C28E758D00758B007563007554CF
:104B710001755300D28EE55D240875F00984AFF00C
:104B81007E00EF4E6003024C0CE56C6013AE55AF36
:104B9100567409126AA190001AEEF0A3EFF0800F8B
:104BA10090001CE0F8A3E090001AC8F0A3C8F090B0
:104BB100001AE0FEA3E0FFEF4E600B7C817DB8128E
:104BC100698F8E518F5290001CE4F0A3F0AE51AF6B
:104BD100527428BE00039F5010E5622FFF50010E52
:104BE10074011200398E518F528552629000DDE0BE
:104BF100A851B8000DD395524008E552900062F0DB
:104C010080099000DDE014900062F0E55D640B60C6
:104C110005E55DB41D099000C6E060031224119002
:104C21000060E0655D6007900061E0B55D03756E51
:104C310000A209B35006A208B3B34003024CE590A9
:104C41000092E0B40173900114E0B40214120D1942
:104C510090007FE075F0BEA4FFAEF08E5B8F5C80AC
:104C610056E56675F00A84FF7E0090058C120048B7
:104C7100E0F55A755900AE59AF5A9000B7E0126A83
:104C8100A174648E048F05FF126A918C5B8D5CE5C3
:104C91005C90001EF0AE59AF5A900090E0126AA1EC
:104CA10074648E048F05FF126A9174BE8C068D07A1
:104CB100126AA18E5B8F5C8017900090E075F0BE48
:104CC100A4FFAEF08E5B8F5C9000B7E090001EF009
:104CD100E560C394CC5006E55C455B70028003122D
:104CE100414DD209E56CB40106E55D640B600280BB
:104CF1000C756F019000647401F0756C00E56C60D7
:104D010003024DDC9000D9E0600D90007EE0A851D7
:104D1100B800069552400280589000D9E0B402379D
:104D210090004DE0655D602790004EE0655D601F7D
:104D310090004FE0655D6017900050E0655D600F89
:104D4100900051E0655D6007900052E0B55D03752C
:104D51006F03756B00800CC200756B00900027E437
:104D6100F0A3F090007EE060067409900063F0808B
:104D71006A90004DE0B55D0B756F019000647401A0
:104D8100F0805890004EE0B55D0B756F0174029094
:104D91000064F0804690004FE0B55D0B756F0174C3
:104DA10003900064F08034900050E0B55D0B756FA6
:104DB100017404900064F08022900051E0B55D0B15
:104DC100756F017405900064F08010900052E0B599
:104DD1005D09756F017406900064F0A206B3920438
:104DE100A206B330B601B35003024F29756D01908D
:104DF10000B9E0B43D13A206B34008E5B54404F59B
:104E0100B58006E5B554FBF5B5A224400575FFA0B4
:104E1100D224E5B54401F5B5741F900076F0A206E1
:104E21009204E55DD3944A4014D208E55DD3946EB3
:104E3100400B7404900063F0D21D755D469000E153
:104E4100E0B40107E569C3941440028009123CA053
:104E51007413900063F0E569C394415009740E9096
:104E61000063F0123CA090006BE0FE900067E0C38D
:104E71009E4009900067E0D39408400974FB9000BC
:104E810063F0123CA0900070E06015900070E0FEAD
:104E910090006AE06E600974FE900063F0123CA01D
:104EA10090089FE06006900111E06002807A740131
:104EB1009000D5F090089FE0906384F828287380D3
:104EC100188016A2A3400674029000D5F0800AA2B1
:094ED100A4400674029000D5F023
:0C638400024EC0024EC2024EC4024ED0B7
:104EDA009000D5E0B40105A223B340028019D22381
:104EEA00123CA01204D574019000D5F0123310D2EE
:104EFA0020741B900063F09000D5E0B40206A22350
:104F0A00B3B340028019C223123CA01205B6740240
:104F1A009000D5F0123310D220741B900063F0A2D7
:104F2A001DB3400CC296C295C2A0C297C2A2C2A12A
:104F3A00900111E0600CAE51AF527414BE00059F8F
:104F4A0040028037900099E0906390F82828738097
:104F5A002A8028A2A3B35005A21FB34002800512DB
:104F6A0041B8D21F8015A2A4B35005A21EB34002B5
:0B4F7A0080051241B8D21E80028000AA
:10639000024F59024F5B024F5D024F70024F830262
:0263A0004F8527
:104F8500A20BB3B35008900053E0655D6002803614
:104F9500A201B35006A200B3B340028023123470BD
:104FA5001234A09000F2E0B40113A202B34008E568
:104FB500B54480F5B58006E5B5547FF5B575A70010
:104FC500C20BD20CD20DA20CB3B35008900054E022
:104FD500655D60028036A201B35006A200B3B340FE
:104FE5000280231234701234AB9000F2E0B4011346
:104FF500A202B34008E5B54480F5B58006E5B55491
:105005007FF5B575A700D20BC20CD20DA20DB3B3B7
:105015005008900055E0655D60028036A201B350EE
:1050250006A200B3B3400280231234701234B69046
:1050350000F2E0B40113A202B34008E5B54480F5DF
:10504500B58006E5B5547FF5B575A700D20BD20C32
:10505500C20DA20BB3B35008900056E0655D600227
:105065008036A201B35006A200B3B34002802312DA
:1050750034701234C19000F2E0B40113A202B340BF
:1050850008E5B54480F5B58006E5B5547FF5B575F9
:10509500A700C20BD20CD20DA20CB3B350089000DE
:1050A50057E0655D60028036A201B35006A200B3E9
:1050B500B3400280231234701234CC9000F2E0B475
:1050C5000113A202B34008E5B54480F5B58006E5B5
:1050D500B5547FF5B575A700D20BC20CD20DA20D44
:1050E500B3B35008900058E0655D60028036A201B8
:1050F500B35006A200B3B3400280231234701234B9
:10510500D79000F2E0B40113A202B34008E5B5441C
:1051150080F5B58006E5B5547FF5B575A700D20BCA
:10512500D20CC20DE56F9063A2F82828730257824E
:045135009000F9E00D
:0663A200025132025135E8
:105139009063E1F8282873121DB38012121DB38001
:0E5149000D121E3D8008121EE98003121EE9A1
:0F63E10002514002514502514A02514F0251549C
:10515700756F0202578212201512212C12244690D5
:10516700088CE0FEA3E0FF740A126AA190001AE01F
:10517700FCA3E0FD74098F02FF126A918D078C036F
:105187008E048A058B0612698F900890EEF0A3EFC4
:10519700F09000E2E0B401087428BE00059F4002C9
:1051A700800D7428900890F8E4F0E8A3F0801B9035
:1051B7000890E0FEA3E0FF74F0BE00039F500B745D
:1051C700F0900890F8E4F0E8A3F0E5357003753542
:1051D70001900890E0FEA3E0FFE5352FFF50010E98
:0F51E700900890EEF0A3EFF0756F03900064E076
:0363A80002515D42
:1051F6009063F0F82828738034A22D4003756F0A57
:10520600802BA22D4003756F0B8022A22D400375C3
:105216006F0C8019A22D4003756F0D8010A22D40D2
:0D52260003756F0E8007A22D4003756F0FFA
:1063F0000251FD0251FF02520802521102521A02CA
:05640000522302522CA2
:105233000257829006D3E060077401F50812256DCA
:10524300900112E0B40114900113E0A851B80004D6
:1052530095525007E55EC3955F400280097415902F
:105263000063F00252EA9000C7E0D39402403F90FB
:10527300009BE02403A851B8000495525009900004
:105283009DE0D3956050028008D2017408900063BA
:10529300F090009BE0A851B80005D39552500B90B5
:1052A300009DE02403C395605002C2018039900041
:1052B3009BE02403A851B8000495525007E55EC350
:1052C300955F40028008D2017408900063F090005B
:1052D3009BE0A851B80005D395525009E55F240F10
:1052E300C3955E5002C2019000E1E07007E569C317
:1052F300941440028002D2019000D6E0B40102D29D
:1053030001A2014005756F04800A756F1090002794
:0B531300E4F0A3F00257829000C7E016
:0663AB0002523602531AF3
:10531E00906405F8282873120E038012120E038073
:0E532E000D120FB1800812106380031210637D
:0F64050002532502532A02532F025334025339F4
:10533C009006D7E060077402F50812256D756F05AD
:10534C000257821211A3756F069006DBE06007749A
:10535C0003F50812256D9006DFE060077404F5086C
:10536C0012256D02578290001EE06006A203B3B3B3
:10537C004002801D90001EE02528FFAE2750010E34
:10538C008E278F28E55DD39406500690001EE014FE
:10539C00F01213E9756F079006E3E060077405F5EA
:1053AC000812256D9006E7E060077406F5081225D3
:1053BC006D025782900114E0B40203120D91121881
:1053CC0019756F089006EBE060077407F508122555
:1053DC006D025782121BD5A20BB35005A20CB34021
:1053EC00028006D20BD20CD20D756F1002578202BE
:1053FC005782900037E0C394465008C2967446908A
:10540C000037F0900059E0B4011DE535240AF5355C
:10541C00900890E0FEA3E0FF740A2FFF50010E905D
:10542C000890EEF0A3EFF085355A75590090004DB9
:10543C00E0F5721234E2E55C900037F090000CE578
:10544C0059F0A3E55AF0E572900038F0C20F9008BD
:10545C0090E0F559A3E0F55A90004DE0F572123446
:10546C00E2E55C900035F0900000E559F0A3E55AB8
:10547C00F0E572900036F0C20E756F030257829001
:10548C00003BE0C3944650139000E2E0B40104C228
:10549C00968002C295744690003BF090005AE0B49E
:1054AC00011DE535240AF535900890E0FEA3E0FFD8
:1054BC00740A2FFF50010E900890EEF0A3EFF085C8
:1054CC00355A75590090004EE0F5721234E2E55CE5
:1054DC0090003BF090000EE559F0A3E55AF0E57210
:1054EC0090003CF0C211900890E0F559A3E0F55AF9
:1054FC0090004EE0F5721234E2E55C900039F090C9
:10550C000002E559F0A3E55AF0E57290003AF0C2BA
:10551C0010756F0302578290003FE0C394465013FE
:10552C009000E2E0B40104C2968002C2A0744690DE
:10553C00003FF090005BE0B4011DE535240AF53521
:10554C00900890E0FEA3E0FF740A2FFF50010E902C
:10555C000890EEF0A3EFF085355A75590090004F86
:10556C00E0F5721234E2E55C90003FF0900010E53B
:10557C0059F0A3E55AF0E572900040F0C213900880
:10558C0090E0F559A3E0F55A90004FE0F572123413
:10559C00E2E55C90003DF0900004E559F0A3E55A7B
:1055AC00F0E57290003EF0C212756F0302578290C4
:1055BC000043E0C3944650139000E2E0B40104C2EF
:1055CC00968002C2977446900043F090005CE0B461
:1055DC00011DE535240AF535900890E0FEA3E0FFA7
:1055EC00740A2FFF50010E900890EEF0A3EFF08597
:1055FC00355A755900900050E0F5721234E2E55CB2
:10560C00900043F0900012E559F0A3E55AF0E572D2
:10561C00900044F0C215900890E0F559A3E0F55ABB
:10562C00900050E0F5721234E2E55C900041F0908D
:10563C000006E559F0A3E55AF0E572900042F0C27D
:10564C0014756F03025782900047E0C394465013C1
:10565C009000E2E0B40104C2968002C2A2744690AB
:10566C000047F090005DE0B4011DE535240AF535E6
:10567C00900890E0FEA3E0FF740A2FFF50010E90FB
:10568C000890EEF0A3EFF085355A75590090005153
:10569C00E0F5721234E2E55C900047F0900014E5FE
:1056AC0059F0A3E55AF0E572900048F0C217900843
:1056BC0090E0F559A3E0F55A900051E0F5721234E0
:1056CC00E2E55C900045F0900008E559F0A3E55A3E
:1056DC00F0E572900046F0C216756F030257829087
:1056EC00004BE0C3944650139000E2E0B40104C2B6
:1056FC00968002C2A1744690004BF090005EE0B41C
:10570C00011DE535240AF535900890E0FEA3E0FF75
:10571C00740A2FFF50010E900890EEF0A3EFF08565
:10572C00355A755900900052E0F5721234E2E55C7E
:10573C0090004BF0900016E559F0A3E55AF0E57295
:10574C0090004CF0C219900890E0F559A3E0F55A7E
:10575C00900052E0F5721234E2E55C900049F09052
:10576C00000AE559F0A3E55AF0E57290004AF0C240
:06577C0018756F038000A8
:1063B10002534F0253720253C00253E00253FB02D5
:1063C10053FE02548B0255230255BB02565302560B
:0463D100EB02578202
:10578200900035E0B55D73A20E404F900000E0FE40
:10579200A3E0FFEF4E6021AE55AF56900000E0FC53
:1057A200A3E0FD120003740A8E048F05FF126A91B2
:1057B200900000ECF0A3EDF0900036E0601A90004B
:1057C20000E0FEA3E0FFAC55AD56EF2DFDEE3CFC34
:1057D200900000ECF0A3EDF0D20EAE53AF54900067
:1057E20000E0FCA3E0FDEFC39DEE9C400D1241FFE3
:1057F200D296C20E74C8900035F0A20EB3B3500711
:10580200900035E0B55D02800D1241FFD29674C85A
:10581200900035F0C20E900037E0B55D70A20F40E7
:105822004F90000CE0FEA3E0FFEF4E6021AE55AFBB
:105832005690000CE0FCA3E0FD120003740A8E04F3
:105842008F05FF126A9190000CECF0A3EDF090002E
:1058520038E0601A90000CE0FEA3E0FFAC55AD56B4
:10586200EF2DFDEE3CFC90000CECF0A3EDF0D20F1E
:10587200AE53AF5490000CE0FCA3E0FDEFC39DEEED
:105882009C400AC2967446900037F0C20FA20FB332
:10589200B35007900037E0B55D02800AC2967446A5
:1058A200900037F0C20F900039E0B55D7EA2104043
:1058B2004F900002E0FEA3E0FFEF4E6021AE55AF35
:1058C20056900002E0FCA3E0FD120003740A8E046D
:1058D2008F05FF126A91900002ECF0A3EDF09000A8
:1058E2003AE0601A900002E0FEA3E0FFAC55AD562C
:1058F200EF2DFDEE3CFC900002ECF0A3EDF0D21097
:10590200AE53AF54900002E0FCA3E0FDEFC39DEE66
:105912009C40181241FF9000E2E0B40104D296804C
:1059220002D295C21074C8900039F0A210B3B350DD
:1059320007900039E0B55D0280181241FF9000E245
:10594200E0B40104D2968002D29574C8900039F076
:10595200C21090003BE0B55D7BA211404F90000E5B
:10596200E0FEA3E0FFEF4E6021AE55AF5690000E71
:10597200E0FCA3E0FD120003740A8E048F05FF12FF
:105982006A9190000EECF0A3EDF090003CE0601AFA
:1059920090000EE0FEA3E0FFAC55AD56EF2DFDEEFC
:1059A2003CFC90000EECF0A3EDF0D211AE53AF54DC
:1059B20090000EE0FCA3E0FDEFC39DEE9C4015902D
:1059C20000E2E0B40104C2968002C29574469000DF
:1059D2003BF0C211A211B3B3500790003BE0B55D9A
:1059E2000280159000E2E0B40104C2968002C295E2
:1059F200744690003BF0C21190003DE0B55D7EA27E
:105A020012404F900004E0FEA3E0FFEF4E6021AE93
:105A120055AF56900004E0FCA3E0FD120003740AA7
:105A22008E048F05FF126A91900004ECF0A3EDF052
:105A320090003EE0601A900004E0FEA3E0FFAC5547
:105A4200AD56EF2DFDEE3CFC900004ECF0A3EDF022
:105A5200D212AE53AF54900004E0FCA3E0FDEFC3BA
:105A62009DEE9C40181241FF9000E2E0B40104D286
:105A7200968002D2A0C21274C890003DF0A212B366
:105A8200B3500790003DE0B55D0280181241FF90CF
:105A920000E2E0B40104D2968002D2A074C8900061
:105AA2003DF0C21290003FE0B55D7BA213404F90E3
:105AB2000010E0FEA3E0FFEF4E6021AE55AF56901E
:105AC2000010E0FCA3E0FD120003740A8E048F05AF
:105AD200FF126A91900010ECF0A3EDF0900040E00C
:105AE200601A900010E0FEA3E0FFAC55AD56EF2D1A
:105AF200FDEE3CFC900010ECF0A3EDF0D213AE539F
:105B0200AF54900010E0FCA3E0FDEFC39DEE9C407B
:105B1200159000E2E0B40104C2968002C2A074466D
:105B220090003FF0C213A213B3B3500790003FE0BE
:105B3200B55D0280159000E2E0B40104C2968002D5
:105B4200C2A0744690003FF0C213900041E0B55DE0
:105B52007EA214404F900006E0FEA3E0FFEF4E60ED
:105B620021AE55AF56900006E0FCA3E0FD12000303
:105B7200740A8E048F05FF126A91900006ECF0A35E
:105B8200EDF0900042E0601A900006E0FEA3E0FF14
:105B9200AC55AD56EF2DFDEE3CFC900006ECF0A3AB
:105BA200EDF0D214AE53AF54900006E0FCA3E0FD3A
:105BB200EFC39DEE9C40181241FF9000E2E0B40159
:105BC20004D2968002D297C21474C8900041F0A207
:105BD20014B3B35007900041E0B55D028018124142
:105BE200FF9000E2E0B40104D2968002D29774C81A
:105BF200900041F0C214900043E0B55D7BA21540D5
:105C02004F900012E0FEA3E0FFEF4E6021AE55AFD1
:105C120056900012E0FCA3E0FD120003740A8E0409
:105C22008F05FF126A91900012ECF0A3EDF0900044
:105C320044E0601A900012E0FEA3E0FFAC55AD56BE
:105C4200EF2DFDEE3CFC900012ECF0A3EDF0D2152E
:105C5200AE53AF54900012E0FCA3E0FDEFC39DEE03
:105C62009C40159000E2E0B40104C2968002C29703
:105C72007446900043F0C215A215B3B350079000CA
:105C820043E0B55D0280159000E2E0B40104C296E3
:105C92008002C2977446900043F0C215900045E01E
:105CA200B55D7EA216404F900008E0FEA3E0FFEF34
:105CB2004E6021AE55AF56900008E0FCA3E0FD1205
:105CC2000003740A8E048F05FF126A91900008EC9B
:105CD200F0A3EDF0900046E0601A900008E0FEA309
:105CE200E0FFAC55AD56EF2DFDEE3CFC900008EC0C
:105CF200F0A3EDF0D216AE53AF54900008E0FCA32F
:105D0200E0FDEFC39DEE9C40181241FF9000E2E0DF
:105D1200B40104D2968002D2A2C21674C890004581
:105D2200F0A216B3B35007900045E0B55D028018AB
:105D32001241FF9000E2E0B40104D2968002D2A2A6
:105D420074C8900045F0C216900047E0B55D7BA292
:105D520017404F900014E0FEA3E0FFEF4E6021AE2B
:105D620055AF56900014E0FCA3E0FD120003740A44
:105D72008E048F05FF126A91900014ECF0A3EDF0EF
:105D8200900048E0601A900014E0FEA3E0FFAC55DA
:105D9200AD56EF2DFDEE3CFC900014ECF0A3EDF0BF
:105DA200D217AE53AF54900014E0FCA3E0FDEFC352
:105DB2009DEE9C40159000E2E0B40104C296800280
:105DC200C2A27446900047F0C217A217B3B350079D
:105DD200900047E0B55D0280159000E2E0B4010456
:105DE200C2968002C2A27446900047F0C217900089
:105DF20049E0B55D7EA218404F90000AE0FEA3E0A4
:105E0200FFEF4E6021AE55AF5690000AE0FCA3E0D2
:105E1200FD120003740A8E048F05FF126A9190002E
:105E22000AECF0A3EDF090004AE0601A90000AE05C
:105E3200FEA3E0FFAC55AD56EF2DFDEE3CFC90000D
:105E42000AECF0A3EDF0D218AE53AF5490000AE082
:105E5200FCA3E0FDEFC39DEE9C40181241FF9000B1
:105E6200E2E0B40104D2968002D2A1C21874C890B2
:105E72000049F0A218B3B35007900049E0B55D02A3
:105E820080181241FF9000E2E0B40104D296800231
:105E9200D2A174C8900049F0C21890004BE0B55DE1
:105EA2007BA219404F900016E0FEA3E0FFEF4E6088
:105EB20021AE55AF56900016E0FCA3E0FD120003A0
:105EC200740A8E048F05FF126A91900016ECF0A3FB
:105ED200EDF090004CE0601A900016E0FEA3E0FFA7
:105EE200AC55AD56EF2DFDEE3CFC900016ECF0A348
:105EF200EDF0D219AE53AF54900016E0FCA3E0FDD2
:105F0200EFC39DEE9C40159000E2E0B40104C296FE
:105F12008002C2A1744690004BF0C219A219B3B319
:105F2200500790004BE0B55D0280159000E2E0B4AE
:105F32000104C2968002C2A1744690004BF0C219BD
:105F42009000E4E0B40202800302606A900078E00C
:105F5200D395655064900078E0F4042565FE9000C6
:105F6200E7E08E00F5F0E884FF7E008F72EFC394C5
:105F720010500CEF8572F0A4FDACF08D72800375A9
:105F820072FF900078E0D39572400B900078E0C3E6
:105F92009572F5708003757000900102E0D39570E0
:105FA2004006900102E0F570900103E0C395705045
:105FB20006900103E0F5708071900078E0C395656A
:105FC200FE9000E7E08E00F5F0E884FF7E008F721D
:105FD200EFC39410500CEF8572F0A4FDACF08D72FB
:105FE20080037572FF85725A755900900078E0251A
:105FF2005AFFAE5950010E8E598F5A74FFBE0009D6
:10600200D39F4005855A7080037570FF900102E0AE
:10601200D395704006900102E0F570900103E0C351
:1060220095705006900103E0F570A203B3B3500DD2
:10603200900079E0FE9000EFE0D39E5002800E7453
:1060420007900063F0E5B554BFF5B5801B75A71046
:10605200E5CDC395704008E5B554BFF5B58006E5BA
:10606200B54440F5B575A7009000FFE0605E900171
:1060720009E0A851B8000495525017900108E0A811
:1060820051B8000ED39552400990010AE0D39560B1
:106092004002801D75A710E5CDC394BF4008E5B549
:1060A20054EFF5B58006E5B54410F5B575A7008047
:1060B2001B75A710E5CDC394404008E5B554EFF534
:1060C200B58006E5B54410F5B575A700900100E06E
:1060D200605E90010CE0A851B800049552501790F0
:1060E200010BE0A851B8000ED39552400990010D62
:1060F200E0D395604002801D75A710E5CDC394BF23
:106102004008E5B554DFF5B58006E5B54420F5B5A0
:1061120075A700801B75A710E5CDC394404008E524
:10612200B554DFF5B58006E5B54420F5B575A70091
:10613200E56EC39409500AA2EDB34005C2ED122ADE
:1061420007AE53AF547414C39F741E9E400C90004C
:1061520077E0C3945A4003026345A208B340091290
:106162003CA07406900063F0A20AB3500EE560D31F
:1061720094334007E560C394CC4002804A900114F6
:10618200E0B40214120D1990007FE075F050A4FFE4
:10619200AEF08E5B8F5C800F900090E075F050A4A3
:1061A200FFAEF08E5B8F5CE55C455B601AA224401B
:1061B2000575FFA0D224E5B54401F5B5741F900022
:1061C20076F012414DD20A900077E0D39401400755
:1061D200E560C3941A40028002C20A9006D3E060CE
:1061E200077401F50812256D9006D7E06007740266
:1061F200F50812256D9006DBE060077403F50812BE
:10620200256D9006DFE060077404F50812256D9095
:1062120006E3E060077405F50812256D9006E7E0D5
:1062220060077406F50812256D9006EBE0600774AE
:1062320007F50812256D900077E0C3945A5026E5C1
:106242006EB40909900077E004F0756E0090007753
:10625200E0B45A0FA224400575FFA0D224E5B5444C
:1062620001F5B5803BE56EB40903756E0075540007
:10627200755300758D00758B00756300900076E094
:10628200C3942E5008900076E004F08006742E909D
:106292000076F0900076E0B42E06E5B554FEF5B532
:1062A200900077E0D394014007E569C3944140022E
:1062B2008009740E900063F0123CA090089FE06089
:1062C20006900111E06002807A74019000D5F0908E
:1062D200089FE09063D5F828287380188016A2A33F
:1062E200400674029000D5F0800AA2A4400674020F
:0462F2009000D5F053
:0C63D5000262DC0262DE0262E00262ECA6
:1062F6009000D5E0B40105A223B340028019D22351
:10630600123CA01204D574019000D5F0123310D2BD
:1063160020741B900063F09000D5E0B40206A2231F
:10632600B3B340028019C223123CA01205B6740210
:106336009000D5F0123310D220741B900063F00247
:0263460047927C
:106414000000010001400160018001A001C001E011
:1064240002000300039603B603D603F40400050038
:106434000512052405360548055A056C057E0590A8
:1064440005A805C005DE0600061406280646066EE5
:1064540006AE05CF00FF013F015F017F019F01BF31
:1064640001DF01FF02FF039503B503D503F303FF27
:1064740004FF05110523053505470559056B057D01
:10648400058F05A705BF05CE05F1061306270645AA
:10649400066D06AD06ED05DD0FAA0FA50F9F0F9A39
:1064A4000F940F8D0F870F800F780F710F680F6097
:1064B4000F570F4E0F450F3B0F300F250F1A0F0EBE
:1064C4000F020EF50EE80EDB0ECC0EBE0EAE0E9FC6
:1064D4000E8E0E7D0E6C0E5A0E470E340E200E0CD0
:1064E4000DF70DE20DCB0DB50D9D0D850D6D0D5404
:1064F4000D3A0D200D050CE90CCE0CB10C940C7664
:106504000C580C3A0C1B0BFB0BDB0BBB0B9A0B79DB
:106514000B570B350B130AF10ACE0AAB0A870A6430
:106524000A400A1C09F809D409B0098C096709430F
:10653400091F08FB08D608B2088E086A0846082313
:1065440007FF07DC07B9079607730751072F070DE5
:1065540006EC06CA06AA068906690649062A060A38
:1065640005EC05CD05B0059205750558053C0520DB
:10657400050504EA04CF04B5049C048204690451AB
:1065840004390422040B03F403DE03C803B2039D9D
:10659400038903750361034D033B032803160304B6
:1065A40002F202E102D102C002B002A00291028210
:1065B4000273026502570249023C022F02220216AC
:1065C400020901FD01F201E601DB01D001C601BBB4
:1065D40001B101A7019D0194018B01820179017030
:1065E400016801600158015001480141013901323B
:1065F400012B0125011E01180111010B010500FFEA
:1066040000FA0FA60FA00F990F920F8B0F840F7C27
:106614000F740F6B0F620F580F4E0F430F380F2C70
:106624000F1F0F120F050EF70EE80ED80EC80EB787
:106634000EA50E930E800E6C0E580E420E2C0E15E7
:106644000DFD0DE40DCB0DB10D950D790D5D0D3FD7
:106654000D200D010CE10CC00C9E0C7C0C590C356A
:106664000C100BEA0BC40B9E0B760B4F0B260AFD8A
:106674000AD40AAA0A800A550A2A09FF09D409A8D1
:10668400097C0950092508F908CD08A10875084AAC
:10669400081E07F307C8079D07730749072006F775
:1066A40006CE06A6067E06570630060A05E405BF92
:1066B400059B057705540532051004EF04CE04AE9E
:1066C400048F047104530435041903FD03E203C762
:1066D40003AD0394037B0363034B0334031E0308DA
:1066E40002F302DE02CA02B602A30291027F026D25
:1066F400025C024C023C022C021D020E020001F25A
:1067040001E401D701CA01BE01B101A6019A018FBA
:106714000185017A01700166015D0153014A01415D
:10672400013901310129012101190112010B01046F
:1067340000FD00F700F000EA00E400DE00D900D319
:1067440000CE00C900C400BF00BA00B500B100AD5E
:1067540000A800A400A0009C009900950091008E60
:0C676400008A008700840081007E007B1A
:10009E00754600900896E4F0A3F0753000752F00B9
:1000AE00754C00754D00C228D22A90089FE0600260
:1000BE00D22074FE900898F8E4F0E8A3F074FE9055
:1000CE00089CF8E4F0E8A3F074FE90089AF8E4F0C7
:1000DE00E8A3F0745A9008BEF0745A9008BFF0D29C
:1000EE002BC226C22DC22CC22722750B00750A0008
:1000FE00AE0AAF0BAC08AD09EDC39FEC9E40167473
:10010E00FF126A8175CF01780B740126F650041820
:10011E00E436F650DB22C2AF75D904758F0375B77E
:10012E00A575B7F190F800E4F0758F0175B7A57558
:10013E00B7F1E52690F800F075B7A575B7F190F810
:10014E0001E4F075B7A575B7F19008B2E090F8022A
:10015E00F075B7A575B7F19008B6E090F803F07595
:10016E00B7A575B7F19008B3E090F804F075B7A590
:10017E0075B7F19008B4E090F805F075B7A575B7AE
:10018E00F19008B5E090F806F075B7A575B7F19047
:10019E0008B7E090F807F0758F0075D944D2AF22FA
:1001AE0090005FE0B4AB61C2AF75D90475B622752D
:1001BE00F522758F0375B7A575B7F1740090F6002B
:1001CE00F0758F01755A00755900AE59AF5A7413F8
:1001DE00BE00279F402475B7A575B7F190089E12F3
:1001EE000048E0FC90F600120048ECF0785A7401DA
:1001FE0026F6500418E436F650D0758F0075F511BA
:10020E0075B62075D944D2AF22C2AF75F52275D915
:10021E0004755A00755900AE59AF5A7413BE0022B8
:10022E009F401F90F600120048E493FC90089E1227
:10023E000048ECF0785A740126F6500418E436F6AD
:10024E0050D575D94475F511D2AF2290005FE0B448
:10025E00AA028003020396C2AF75D90475B6227541
:10026E00F522758F0375B7A575B7F1740090EE0082
:10027E00F075B7A575B7F1740090F000F075B7A5DD
:10028E0075B7F1740090F200F075B7A575B7F174FB
:10029E000090F400F0758F01755A00755900AE5933
:1002AE00AF5A74FFC39F74019E402475B7A575B7EE
:1002BE00F190008C120048E0FC90EE00120048EC29
:1002CE00F0785A740126F6500418E436F650CF75BD
:1002DE005A00755900AE59AF5A74FFC39F74019EF0
:1002EE00402475B7A575B7F190028C120048E0FC5A
:1002FE0090F000120048ECF0785A740126F6500483
:10030E0018E436F650CF755A00755900AE59AF5AEB
:10031E0074FFC39F74019E402475B7A575B7F19005
:10032E00048C120048E0FC90F200120048ECF078C9
:10033E005A740126F6500418E436F650CF755A005A
:10034E00755900AE59AF5A74FFC39F74019E402475
:10035E0075B7A575B7F190068C120048E0FC90F4C5
:10036E0000120048ECF0785A740126F6500418E496
:10037E0036F650CF758F0075F51175B62075D944C8
:10038E00D2AF743A90078CF02290005FE0B4AA02CC
:10039E0080030204D4C2AF75D90475B62275F52256
:1003AE00758F0375B7A575B7F1740090E600F075FB
:1003BE00B7A575B7F1740090E800F075B7A575B7DD
:1003CE00F1740090EA00F075B7A575B7F17400905E
:1003DE00EC00F0758F01755A00755900AE59AF5A81
:1003EE0074FFC39F74019E402475B7A575B7F19035
:1003FE00008C120048E0FC90E600120048ECF07809
:10040E005A740126F6500418E436F650CF755A0089
:10041E00755900AE59AF5A74FFC39F74019E4024A4
:10042E0075B7A575B7F190028C120048E0FC90E804
:10043E0000120048ECF0785A740126F6500418E4C5
:10044E0036F650CF755A00755900AE59AF5A74FF33
:10045E00C39F74019E402475B7A575B7F190048CA7
:10046E00120048E0FC90EA00120048ECF0785A7452
:10047E000126F6500418E436F650CF755A00755919
:10048E0000AE59AF5A74FFC39F74019E402475B7D6
:10049E00A575B7F190068C120048E0FC90EC0012A6
:1004AE000048ECF0785A740126F6500418E436F63B
:1004BE0050CF758F0075F51175B62075D944D2AF32
:1004CE00743A90078CF022C2AF75D90475F5227577
:1004DE005A00755900AE59AF5A74FFC39F74019EEE
:1004EE00401F90EE00120048E493FC90008C120026
:1004FE0048ECF0785A740126F6500418E436F6509B
:10050E00D4755A00755900AE59AF5A74FFC39F7413
:10051E00019E401F90F000120048E493FC90028C64
:10052E00120048ECF0785A740126F6500418E4369E
:10053E00F650D4755A00755900AE59AF5A74FFC3B0
:10054E009F74019E401F90F200120048E493FC90AD
:10055E00048C120048ECF0785A740126F6500418F8
:10056E00E436F650D4755A00755900AE59AF5A7428
:10057E00FFC39F74019E401F90F400120048E49345
:10058E00FC90068C120048ECF0785A740126F65056
:10059E000418E436F650D475F51175D944D2AF74FB
:1005AE003A90078CF0C22922C2AF75D90475F52294
:1005BE00755A00755900AE59AF5A74FFC39F740136
:1005CE009E401F90E600120048E493FC90008C12AF
:1005DE000048ECF0785A740126F6500418E436F60A
:1005EE0050D4755A00755900AE59AF5A74FFC39F57
:1005FE0074019E401F90E800120048E493FC9002A4
:10060E008C120048ECF0785A740126F6500418E467
:10061E0036F650D4755A00755900AE59AF5A74FF5C
:10062E00C39F74019E401F90EA00120048E493FCA1
:10063E0090048C120048ECF0785A740126F650049F
:10064E0018E436F650D4755A00755900AE59AF5AA3
:10065E0074FFC39F74019E401F90EC00120048E48B
:10066E0093FC90068C120048ECF0785A740126F632
:10067E00500418E436F650D475F51175D944D2AF3E
:10068E00743A90078CF0D22922E54D64046006E599
:10069E009964FF60028031A2284004D2288027E5A9
:1006AE004D600874E6254D900063F0E54C600874CB
:1006BE00F0254C900063F0E54DB4010280FE754DBF
:1006CE0000754C00C2288002C228E54D903280F899
:1006DE00282873754D00E599B4FF03754C01E59913
:1006EE00B4FE03754C02E599B4FD03754C03E59910
:1006FE00B4FC03754C04E599B4FA03754C05E59901
:10070E00B4FB06754D01123CA0E599B4F906754D82
:10071E0004123CA0E599D394E54007E599C394F003
:10072E004002801685994E754D027E017F00E54E82
:10073E00C394E6126AA18E318F32900896E4F0A32C
:10074E00F0E599D394C44007E599C394E64002803E
:10075E002885994E754D0374E5C3954EF532753166
:10076E0000AE31AF32906414126A70E493F87401E3
:10077E0093900896C8F0A3C8F0D299020B77900810
:10078E009EE0700AA221B35005A222B3400280421D
:10079E00900896E0FEA3E0FF74FFBE00039F500991
:1007AE00EFC39446EE94064011900896E0FEA3E047
:1007BE00FFEFD3946DEE94064013900896E0FEA3DF
:1007CE00E0FF90008C120048E599F0800385997344
:1007DE008011900896E0FEA3E0FF90008C12004876
:1007EE00E599F0900896126AAF900896E0FEA3E0A5
:1007FE00FFEFB40106EEB407028003020970900702
:10080E008CE0B43C028003020970A221B35005A211
:10081E0022B340030208E7C29C90089EE090012A92
:10082E00F090089FE0900099F09008A0E09000B939
:10083E00F09008A1E09000E2F09008A2E090008E07
:10084E00F09008A3E09000D4F09008A4E09000F29D
:10085E00F09008A5E09000C6F09008A6E09000E4A5
:10086E00F09008A7E0900114F09008A8E0900178AD
:10087E00F09008A9E0900179F09008AAE090017A32
:10088E00F012356490007AE09000FBF090007BE06F
:10089E009000B2F090007CE09000B3F074AB90004A
:1008AE005FF01201AE74AA90005FF0A229B340056A
:1008BE00120397800312025990005FE4F0900178C2
:1008CE00E0700C900179E0700690017AE060028091
:1008DE0004C2218002D221807EC29C90012AE09027
:1008EE00089EF0900099E090089FF09000B9E0907B
:1008FE0008A0F09000E2E09008A1F090008EE09049
:10090E0008A2F09000D4E09008A3F09000F2E090DE
:10091E0008A4F09000C6E09008A5F09000E4E090E6
:10092E0008A6F0900114E09008A7F074009008A8B3
:10093E00F074009008A9F074009008AAF074AB90BF
:10094E00005FF01201AE74AA90005FF0120259120D
:10095E0003977599FB80FED29C754D00754C007502
:10096E0099FB020B77900896E0FEA3E0FFEF4E7026
:10097E0006859930752F00900896E0FEA3E0FF746F
:10098E00016F4E701BAC2FAD30AA31AB32ED2BFB8D
:10099E00EC3AFA8A068B0790008C120048E599F023
:1009AE00900896126AAF900896E0FEA3E0FF7402DC
:1009BE006F4E7021AC2FAD3074566D4C7006E54EF7
:1009CE0064E660028003123CA0123564854E997570
:1009DE004D00754C00020B77900896E0FEA3E0FFE9
:1009EE0090008C120048E599F0900896126AAF902C
:1009FE000896E0FEA3E0FFAC31AD328F028E038C81
:100A0E00068D07906458126A70E493F9740193FE90
:100A1E00EAD39EEB994009854E99754D00754C00B1
:100A2E00020B77900896E0FEA3E0FF90008C120078
:100A3E0048E599F0900896126AAF900896E0FEA3EA
:100A4E00E0FFEFB40006EEB401028003020B7790D4
:100A5E00006FE0D394C7400B90006FE0C394C8F5CD
:100A6E004F801A90006FE0D39463400B90006FE0BC
:100A7E00C39464F54F800690006FE0F54FE54F7517
:100A8E00F002A4FFAEF08F72EF90008C126AD2EFDC
:100A9E00FCE0FDEC90008F126AD2EDFCE0FDEC2D37
:100AAE00B54F028003020B680FEF90008C126AD2D2
:100ABE00E572FFE0FCEF900090126AD2ECFFE0FCD2
:100ACE00EFC39CB54F028003020B68E57290008E57
:100ADE00126AD2E572FFE0FCEF900091126AD2EC3E
:100AEE00FFE0FCEF2CB54F72E572900092126AD2C5
:100AFE00E0C3954F9008B2F0E572900093126AD25F
:100B0E00E0C3954F9008B3F0E572900096126AD24A
:100B1E00E0C3954F9008B4F0E572900097126AD238
:100B2E00E0C3954F9008B5F0E572900098126AD226
:100B3E00E0C3954F9008B6F0E572900099126AD214
:100B4E00E0C3954F9008B7F01201247599F97464BB
:100B5E00F5097508001200F880FE7599FF7464F5AA
:090B6E00097508001200F880FE70
:0F3280000206E102078C0209730209E6020A3115
:100B770022E54C90328FF8282873020C5C90089677
:100B8700E0FEA3E0FF900065120048E0F5999008A9
:100B970096126AAF900896E0FEA3E0FF74116F4EBD
:100BA7007003754C00020C5C856D99020C5C900813
:100BB70096E0FEA3E0FF90008C120048E0F599EF65
:100BC700B40107EEB40703754C00900896126AAF9C
:070BD700020C5C900897E09E
:0F328F00020B81020B84020BAF020BB5020BDAAC
:100BDE009032E3F82828738552998067855E998054
:100BEE0062856099805D8564998058856699805389
:100BFE00856799804E85689980498569998044906A
:100C0E000028E0F599803CA22AB340077599FAC2F4
:100C1E002A8017A220B3400575990F800B900063B0
:100C2E00E0F599900063E4F0C2208017856A998000
:100C3E0012856599800D856B9980087599FC8003E6
:030C4E00754C00E2
:1032E300020BE5020BEA020BEF020BF4020BF902ED
:1032F3000BFE020C03020C08020C0D020C15020C4F
:0D3303003A020C3F020C44020C49020C4E31
:0B0C5100900896126AAF80031233ED8A
:03329E00020C59C6
:100C5C0022E536255AFFAE5950010E90008C120039
:100C6C0048E0F537E536255AFFAE5950010E0FBF57
:100C7C0000010E90008C120048E0F538853E3AE5F4
:100C8C0037B538058537368041E538D39537401D63
:100C9C00E538C395378539F0A4FFAEF0E53A8E04FC
:100CAC008F05FF126A91ED2537F536801DE537C3A8
:100CBC0095388539F0A4FFAEF0E53A8E048F05FF28
:100CCC00126A91EDF4042537F53622E538D39537C1
:100CDC00401DE538C395378539F0A4FFAEF0E53AF1
:100CEC008E048F05FF126A91ED2537F536801DE5D0
:100CFC0037C395388539F0A4FFAEF0E53A8E048FF2
:100D0C0005FF126A91EDF4042537F5362290009216
:100D1C00E0B40170E56675F00A84FF7E008F36E55D
:100D2C006675F00A84ADF07C008D39753E0A7559F4
:100D3C0005755A24E536C394115005120C5D8006D6
:100D4C009005C1E0F536E53690007FF0E56675F06C
:100D5C000A84FF7E008F36E56675F00A84ADF07C60
:100D6C00008D39753E0A755905755A5AE536C39486
:100D7C00115005120C5D80069005F7E0F536E5364E
:100D8C0090001EF022900092E0B4016AE56675F0C6
:100D9C000A84FF7E008F36E56675F00A84ADF07C20
:100DAC00008D39753E0A755905755A36E536C3946A
:100DBC00115005120C5D80069005D3E0F536853692
:100DCC004AE56675F00A84FF7E008F36E56675F09D
:100DDC000A84ADF07C008D39753E0A755905755A3B
:100DEC0048E536C394115005120C5D80069005E55C
:100DFC00E0F53685364B22E55E75F00484FF7E0007
:100E0C008F36E55E75F00484ADF07C008D39753E4F
:100E1C0004755901755A00E536C3943F5005120C00
:100E2C005D80069001CBE0F536853628752700905D
:100E3C000062E075F020A4FFAEF09000DDE08E04BF
:100E4C008F05FF126A918D369000C5E0D3955E50E8
:100E5C0003020F099000E9E0D3955E4010ED90017C
:100E6C00CC126AD2E0F52A752900020F069000B464
:100E7C00E0D3955E4043E5369001CC126AD2E0F5A2
:100E8C0037E5369001EC126AD2E0F5389000E9E0D3
:100E9C00F404255EF5399000B4E0FE9000E9E0F42E
:100EAC00042EF53AE537B538058537368003120C34
:100EBC00D785362A7529008041E5369001EC126AF7
:100ECC00D2E0F537E53690020C126AD2E0F5389094
:100EDC0000B4E0F404255EF5399000C5E0FE900006
:100EEC00B4E0F4042EF53AE537B53805853736808D
:100EFC0003120CD785362A752900020FB09000EC2E
:100F0C00E0D3955E5011E53690024C126AD2E0F5B2
:100F1C002A752900020FB09000B5E0D3955E5043BE
:100F2C00E53690022C126AD2E0F537E53690024C89
:100F3C00126AD2E0F5389000B5E0F404255EF5397C
:100F4C009000ECE0FE9000B5E0F4042EF53AE537A5
:100F5C00B538058537368003120CD785362A7529A6
:100F6C00008041E53690020C126AD2E0F537E53686
:100F7C0090022C126AD2E0F5389000C5E0F40425FA
:100F8C005EF5399000B5E0FE9000C5E0F4042EF556
:100F9C003AE537B538058537368003120CD78536D8
:100FAC002A752900229000FDE0F53B753E1175591C
:100FBC0002755A00AE51AF52E53B75F00FA4FDAC73
:100FCC00F0EDD39FEC9E4021E53B8E048F05FF1284
:100FDC006A91ED75F010A4FFAEF0E55E75F011842A
:100FEC00FD7C00ED2FF53C800EE55E75F01184FF65
:100FFC007E00EF24F0F53C853C36E55E75F01184FF
:10100C00AFF07E008F39120C5D85363DAE51AF527C
:10101C009000FDE075F00FA4FDACF0EDD39FEC9EBD
:10102C004028755902755A10853C36120C5D853D69
:10103C0037853638AE51AF52E53B8E048F05FF1223
:10104C006ABC8D39853B3A120CD78536287527003A
:10105C00752A64752900229000FDE0F53B753E1160
:10106C00755902755A00AE51AF52E53B75F00FA49D
:10107C00FDACF0EDD39FEC9E4021E53B8E048F053B
:10108C00FF126A91ED75F010A4FFAEF0E56075F0FB
:10109C001184FD7C00ED2FF53C800EE56075F011A0
:1010AC0084FF7E00EF24F0F53C853C36E56075F05E
:1010BC001184AFF07E008F39120C5D85363DAE5138
:1010CC00AF529000FDE075F00FA4FDACF0EDD39F96
:1010DC00EC9E4028755902755A10853C36120C5DF1
:1010EC00853D37853638AE51AF52E53B8E048F05C2
:1010FC00FF126ABC8D39853B3A120CD785362875A0
:10110C002700E56A6017E56AC394FE50109000F161
:10111C00E0B402099000DFE0D3940B50028017AECC
:10112C0027AF28E56A126AA174E78E048F05FF12B7
:10113C006A918C278D289000C7E0B40453E55E7546
:10114C00F00484FF7E008F36E55E75F00484ADF00C
:10115C007C008D39753E04755901755A00E536C30E
:10116C00943F5005120C5D80069001CBE0F536AE35
:10117C0027AF28E536126AA174648E048F05FF121E
:10118C006A91AE27AF28EF2DFDEE3CFC8C278D2805
:10119C00752A6475290022900092E0B40146E56638
:1011AC0075F00A84FF7E008F36E56675F00A84AD13
:1011BC00F07C008D39753E0A755905755A00E53677
:1011CC00C394115005120C5D800690059DE0F53618
:1011DC00AE29AF2AE5362FFF50010E7464126AE473
:1011EC008E298F2A900093E0B40146E56775F00ACA
:1011FC0084FF7E008F36E56775F00A84ADF07C00C5
:10120C008D39753E0A755905755A6CE536C39411BE
:10121C005005120C5D8006900609E0F536AE29AF3C
:10122C002AE5362FFF50010E7464126AE48E298F62
:10123C002A9000A2E0B40249E569C3944175F00517
:10124C0084FF7E008F36E56975F00584ADF07C0077
:10125C008D39753E05755906755A00E536C39413DC
:10126C005005120C5D800690069FE0F536AE29AF56
:10127C002AE5362FFF50010E7464126AE48E298F12
:10128C002A9000E4E0B402028003021342E55E758A
:10129C00F01584FF7E008F36E55E75F01584ADF099
:1012AC007C008D39753E15755903755AF4E536C3B6
:1012BC00940B5005120C5D800690048BE0F536E51E
:1012CC003675F0FFA4FFAEF09000E5E08E048F05BC
:1012DC00FF126A91ED900078F0E56575F078A4FF47
:1012EC00AEF074FF8E048F05FF126A918C598D5AE3
:1012FC0074028C068D071200398F36AC59AD5A74B6
:10130C0004FF126ABC8D39753E04755906755A284E
:10131C00E536C3941D5005120C5D80069006D1E095
:10132C00F536AE29AF2AE5362FFF50010E74641244
:10133C006AE48E298F2A900091E0B4025DE5607515
:10134C00F064A4FFAEF074081200398E5B8F5C74ED
:10135C00058E048F05FF126A918D36AE5BAF5C74FF
:10136C00058E048F05FF126ABC8D39753E057559C3
:10137C0005755ADEE536C394135005120C5D8006D4
:10138C0090067DE0F536AE29AF2AE5362FFF5001E9
:10139C000E7464126AE48E298F2A9000D3E0703C9C
:1013AC00900062E075F00584FF7E008F369000623D
:1013BC00E075F00584ADF07C008D39753E057559EE
:1013CC0005755AC0E536C3941D5005120C5D800698
:1013DC00900669E0F536E536900080F02290009A90
:1013EC00E0B401179008B9E0252AFFAE2950010E90
:1013FC009000EEE0126AE48E298F2A900112E0B47C
:10140C000114900113E0A851B8000495525007E55F
:10141C005EC3955F400280139000BCE0252AFFAEAE
:10142C002950010E8E298F2A02181890009AE0B4C8
:10143C000306A226B3B3400280509008C2E070109D
:10144C009008BCE0C39405A851B800069552400220
:10145C0080109000BCE0252AFFAE2950010E8E2989
:10146C008F2A9008C2E0600D9008BCE0A851B8002B
:10147C00069552400280109000BCE0252AFFAE2950
:10148C0050010E8E298F2A021818900094E0B40295
:10149C00028003021818900097E0602FE566D39441
:1014AC0046402890001FE0FEA3E0FF9000D2E075BC
:1014BC00F003A4FDACF0EFD39DEE9C400E9000F633
:1014CC00E0A851B80005D3955250030218189000AB
:1014DC00C7E0B40302800302167C85605A7559007C
:1014EC0090009EE0A851B800049552500E90009FB9
:1014FC00E0A859B80005D3955A5003021679E56057
:10150C0075F002A4FFAEF074158E048F05FF126AFD
:10151C00918C068D0790061C120048FEE0FFEE90A1
:10152C000096E0FEEF8E0088F0A4FFAEF074648E9F
:10153C00048F05FF126A918C598D5A900062E075E8
:10154C00F018A4FFAEF09000DDE08E048F05FF12C2
:10155C006A918C068D07900634120048AE59AF5A2A
:10156C00E0126AA174648E048F05FF126A918C5983
:10157C008D5AE564A859B80077D3955A4072E56442
:10158C00C3955AFFE49559FE8E598F5A7428BE00A4
:10159C00039F500C755A28755900740D900063F018
:1015AC00AE59AF5A900097E0126AA174288E048F3E
:1015BC0005FF126A918C598D5AAE27AF28740A8E8A
:1015CC00048F05FF126A918D068C07AC59AD5ACF6A
:1015DC00CECF120003740A8E048F05FF126A918C11
:1015EC00598D5AAE27AF28126AEC8E278F28807D32
:1015FC00E564A859B80004955A5072AE59AF5AE533
:10160C0064126AE48E598F5A7428BE00039F500CE2
:10161C00755A28755900740D900063F0AE59AF5A85
:10162C00900097E0126AA174288E048F05FF126A4D
:10163C00918C598D5AAE27AF28740A8E048F05FFF2
:10164C00126A918D068C07AC59AD5ACFCECF1200D1
:10165C0003740A8E048F05FF126A918C598D5AAE51
:10166C0027AF28EF2DFDEE3CFC8C278D2802181897
:10167C009000DFE0855EF0A4FFAEF07405126AA165
:10168C0074071200398E598F5A90009EE0A851B8F9
:10169C0000049552501290009FE075F002A4FDAC2E
:1016AC00F0EFC39DEE9C4003021818E55E75F00B3D
:1016BC0084FF7E0090061C120048FEE0FFEE9000B6
:1016CC0096E0FEEF8E0088F0A4FFAEF074648E04FA
:1016DC008F05FF126A918C598D5A900062E075F05B
:1016EC0018A4FFAEF09000DDE08E048F05FF126AA7
:1016FC00918C068D07900634120048AE59AF5AE013
:10170C00126AA174648E048F05FF126A918C598D34
:10171C005AE564A859B80077D3955A4072E564C36A
:10172C00955AFFE49559FE8E598F5A7428BE0003C2
:10173C009F500C755A28755900740D900063F0AECB
:10174C0059AF5A900097E0126AA174288E048F0545
:10175C00FF126A918C598D5AAE27AF28740A8E04E9
:10176C008F05FF126A918D068C07AC59AD5ACFCEFE
:10177C00CF120003740A8E048F05FF126A918C59E4
:10178C008D5AAE27AF28126AEC8E278F28807DE504
:10179C0064A859B80004955A5072AE59AF5AE56412
:1017AC00126AE48E598F5A7428BE00039F500C7530
:1017BC005A28755900740D900063F0AE59AF5A90C9
:1017CC000097E0126AA174288E048F05FF126A91AB
:1017DC008C598D5AAE27AF28740A8E048F05FF12D0
:1017EC006A918D068C07AC59AD5ACFCECF1200033F
:1017FC00740A8E048F05FF126A918C598D5AAE278C
:10180C00AF28EF2DFDEE3CFC8C278D28229000F2AA
:10181C00E0B4026AE55E75F00884FF7E008F36E561
:10182C005E75F00884ADF07C008D39753E087559F5
:10183C0001755AE0E536C3943F5005120C5D8006E5
:10184C0090028BE0F53685362C752B00AE2BAF2C29
:10185C00AC29AD2A12000374648E048F05FF126A42
:10186C00918C2B8D2C90008FE08C068D07126AA129
:10187C0074648E048F05FF126A918C2B8D2CAE270D
:10188C00AF28AC29AD2A12000374648E048F05FFB7
:10189C00126A918C278D2890008FE08C068D071290
:1018AC006AA174648E048F05FF126A918C278D28AF
:1018BC00A203401DAE51AF527405BE00039F5002EF
:1018CC00D203E560D394CC4008D20174119000632C
:1018DC00F09000F1E0B402089000DFE0640B6002CD
:1018EC008035AE27AF28E56A126AA174E78E048FA3
:1018FC0005FF126A918C278D289000F2E0B4021734
:10190C00AE2BAF2CE56A126AA174E78E048F05FF2B
:10191C00126A918C2B8D2C9000B1E05402601B90BC
:10192C0000A8E0A851B80012D39552400DA203B301
:10193C00B35007E560C3949A40028028AE33AF34AD
:10194C009000A6E075F002A4FDACF0EF2DFDEE3C8E
:10195C00FC74022DFD50010CE560BC0007D39D40CA
:10196C0003754201856034753300E5427003021A39
:10197C005C900104E0C395425003021A4E9001148E
:10198C00E0C394025076E56675F00A84FF7E009001
:10199C00058C120048E0F55A755900AE59AF5A90B3
:1019AC0000A7E0126AA174648E048F05FF126A917D
:1019BC008C5B8D5C900104E004C395428C068D0712
:1019CC00126AA1900104E08E048F05FF126A918CBB
:1019DC005B8D5CAE27AF28EF2DFDEE3CFC8C278D8C
:1019EC00289000F2E0B40212AE2BAF2CAA5BAB5CD9
:1019FC00EF2BFBEE3AFA8A2B8B2C8046900104E0FD
:101A0C0004C39542854AF0A4FFAEF0900104E08E29
:101A1C00048F05FF126A918C5B8D5CAE27AF28EFAB
:101A2C002DFDEE3CFC8C278D289000F2E0B40212C8
:101A3C00AE2BAF2CAA5BAB5CEF2BFBEE3AFA8A2BEE
:101A4C008B2C0542900104E0C39542500375420073
:101A5C009000B1E05401601B9000A5E0A851B800C3
:101A6C0012D39552400DA203B3B35007E55EC39455
:101A7C00CC400280259000A3E075F003A4FFAEF0EB
:101A8C00E53F2FFF50010E74032FFF50010EE55E52
:101A9C00BE0007D39F4003754301855E3FE543704D
:101AAC0003021B8F900105E0C395435003021B8179
:101ABC00900114E0C394025076E56675F00A84FF39
:101ACC007E0090058C120048E0F55A755900AE590D
:101ADC00AF5A9000A4E0126AA174648E048F05FFC3
:101AEC00126A918C5B8D5C900105E004C395438C6C
:101AFC00068D07126AA1900105E08E048F05FF1276
:101B0C006A918C5B8D5CAE27AF28EF2DFDEE3CFC13
:101B1C008C278D289000F2E0B40212AE2BAF2CAAC9
:101B2C005BAB5CEF2BFBEE3AFA8A2B8B2C8046904E
:101B3C000105E004C39543854BF0A4FFAEF0900182
:101B4C0005E08E048F05FF126A918C5B8D5CAE27CD
:101B5C00AF28EF2DFDEE3CFC8C278D289000F2E099
:101B6C00B40212AE2BAF2CAA5BAB5CEF2BFBEE3AA4
:101B7C00FA8A2B8B2C0543900105E0C39543500347
:101B8C00754300900107E02528FFAE2750010E8E0B
:101B9C00278F289000B6E0A827B800049528500994
:101BAC009000B6E0F5287527009000F2E0B4020D25
:101BBC009000B6E0A82BB80006952C400280099046
:101BCC0000B6E0F52C752B00229000F2E0B4010277
:101BDC008003021CE0A203B35003021CDE9000BD84
:101BEC00E0B40168AE27AF28AC51AD5212000374BB
:101BFC003C8E048F05FF126A919000CDE0BC001062
:101C0C009D400D9000CFE0A827B800049528500205
:101C1C00D202AE27AF28AC51AD52120003743C8EE9
:101C2C00048F05FF126A919000CDE0C3940ABC00AA
:101C3C0015D39D40119000CFE0C39405A827B800A0
:101C4C0005D3952850028002C2028068AE27AF28C7
:101C5C00AC51AD5212000374788E048F05FF126ADA
:101C6C00919000CDE0BC00109D400D9000CFE0A8FD
:101C7C0027B8000495285004D2028038AE27AF282C
:101C8C00AC51AD5212000374788E048F05FF126AAA
:101C9C00919000CDE0C3940ABC0015D39D401190E7
:101CAC0000CFE0C39405A827B80005D395285002AF
:101CBC008002C202A202B34019AE27AF289000CE18
:101CCC00E0126AA174648E048F05FF126A918C274E
:101CDC008D288002C202A200B34006A201B3B35009
:101CEC0009900027E4F0A3F08024AE27AF287400FD
:101CFC00D39F74019E400C900027E527F0A3E528A4
:101D0C00F0800B74FF900027F8E4F0E8A3F090004B
:101D1C00BDE0B4011AAE27AF287402126AA18E2757
:101D2C008F28AE2BAF2C7402126AA18E2B8F2C90A5
:101D3C0000D4E0C394034009900088E0C39402509F
:101D4C0035AE27AF28745E126AA1740A8E048F0513
:101D5C00FF126A918C278D289000F2E0B40217AE26
:101D6C002BAF2C745E126AA1740A8E048F05FF12BD
:101D7C006A918C2B8D2CAE27AF287402BE000AD32F
:101D8C009F4006752802752700AE2BAF2C7402BE3F
:101D9C00000AD39F4006752C02752B00900025E598
:101DAC0027F0A3E528F022900062E090038C126AE1
:101DBC00D2E0F540754164900062E0FE9000C8E00E
:101DCC00D39E4037E55E75F00884FF7E008F36E5C4
:101DDC005E75F00884ADF07C008D39753E08755940
:101DEC0003755A96E536C3941F5005120C5D800698
:101DFC00900441E0F5368536418035E55E75F00896
:101E0C0084FF7E008F36E55E75F00884ADF07C00B3
:101E1C008D39753E08755903755AB6E536C3941F4E
:101E2C005005120C5D8006900461E0F53685364154
:101E3C00229000FEE0F53B753E11755904755A0071
:101E4C00AE51AF52E53B75F00FA4FDACF0EDD39F56
:101E5C00EC9E4021E53B8E048F05FF126A91ED75D7
:101E6C00F010A4FFAEF0E55E75F01184FD7C00ED82
:101E7C002FF53C800EE55E75F01184FF7E00EF249B
:101E8C00F0F53C853C36E55E75F01184AFF07E00D4
:101E9C008F39120C5D85363DAE51AF529000FEE08D
:101EAC0075F00FA4FDACF0EDD39FEC9E4028755956
:101EBC0004755A10853C36120C5D853D37853638D5
:101ECC00AE51AF52E53B8E048F05FF126ABC8D39C3
:101EDC00853B3A120CD7853640754164229000FE42
:101EEC00E0F53B753E11755904755A00AE51AF5271
:101EFC00E53B75F00FA4FDACF0EDD39FEC9E4021BB
:101F0C00E53B8E048F05FF126A91ED75F010A4FF6E
:101F1C00AEF0E56075F01184FD7C00ED2FF53C8092
:101F2C000EE56075F01184FF7E00EF24F0F53C8522
:101F3C003C36E56075F01184AFF07E008F39120CE1
:101F4C005D85363DAE51AF529000FEE075F00FA4AA
:101F5C00FDACF0EDD39FEC9E4028755904755A10DA
:101F6C00853C36120C5D853D37853638AE51AF5207
:101F7C00E53B8E048F05FF126ABC8D39853B3A1206
:101F8C000CD78536407541649000F9E0B404799023
:101F9C000062E0FE9000C8E0D39E4037E55E75F02D
:101FAC000884FF7E008F36E55E75F00884ADF07C0A
:101FBC00008D39753E08755903755A96E536C394EC
:101FCC001F5005120C5D8006900441E0F5368536F5
:101FDC00418035E55E75F00884FF7E008F36E55E46
:101FEC0075F00884ADF07C008D39753E0875590389
:101FFC00755AB6E536C3941F5005120C5D800690D9
:10200C000461E0F53685364122900092E0B4013B44
:10201C00E56675F00A84FF7E008F36E56675F00A7A
:10202C0084ADF07C008D39753E0A755905755A12D0
:10203C00E536C394115005120C5D80069005AFE097
:10204C00F536E5412536C39464F541900093E0B430
:10205C00013BE56775F00A84FF7E008F36E56775F6
:10206C00F00A84ADF07C008D39753E0A7559057502
:10207C005A7EE536C394115005120C5D800690060D
:10208C001BE0F536E5412536C39464F541E5402562
:10209C0041F53590009AE0B402109008B8E025356F
:1020AC00FE9000EEE0F4042EF5359000F1E0D394B0
:1020BC00014040E56AC394E7501D74E7C3956AFE7E
:1020CC009008BAE08E00F5F0E884FF7E008F36E5CC
:1020DC00352536F535801CE56AC394E7FE9008BAC1
:1020EC00E08E00F5F0E884FF7E008F36E535C39571
:1020FC0036F535A2034006E5402464F535E535D3C5
:10210C0094644009E535C39464F535800375350056
:10211C009000CAE0C3953550069000CAE0F5352210
:10212C00D20090007EE0A851B800049552503E9029
:10213C00007EE0A851B800049552500375350F90FD
:10214C00007EE004A851B800049552500375350781
:10215C0090007EE02402A851B8000495525002C2AF
:10216C000090007EE060067409900063F0C22D7E42
:10217C00017F009000D0E0126AA19000DFE08E0495
:10218C008F05FF126A91E55EBC0017D39D4013903A
:10219C0000D9E0B40204D22D8002C200740A90006F
:1021AC0063F0900092E0B401099000D1E0C3956611
:1021BC00400280159000E3E0A851B80004955250FD
:1021CC0002C200740B900063F0900092E0B401071F
:1021DC00E566C394644002801D900129E0600D9077
:1021EC000129E0A851B80006955240028008C200AF
:1021FC00740B900063F0A20040037535009001123F
:10220C00E0B40114900113E0A851B80004955250A9
:10221C0007E55EC3955F400280209000BBE0D3943D
:10222C001D400B9000BBE0C3941EF5358003753543
:10223C00007415900063F002231D90009AE0B40323
:10224C0006A226B3B3400302231D9008BCE0C3943E
:10225C0005A851B80004955250069008C2E06002DF
:10226C00801D9000BBE0D3941D400B9000BBE0C3DD
:10227C00941EF5358003753500740C900063F09056
:10228C0008BCE0A851B80004955250069008C2E072
:10229C007002801D9000BBE0D3941D400B9000BBDE
:1022AC00E0C3941EF5358003753500740C90006303
:1022BC00F09008BCE0A851B8000495525031900041
:1022CC00D9E0B40228D22D9008C1E0FE9008C2E0FB
:1022DC00D39E50069008C2E0700280099008C1E4B9
:1022EC00F0C22D80069008C1E004F08002C200907C
:1022FC0008BCE02405A851B8000495525013900076
:10230C00D9E0B4020A9008C2E07002D22D8002C259
:10231C0000A22CB3401D9000BBE0D3941D400B9049
:10232C0000BBE0C3941EF535800375350074109026
:10233C000063F085356B9000BBE0D3941D40189082
:10234C000089E02535FE900062E075F01E84FC7F6C
:10235C0000EE2CF5358049900063E0640C600F9022
:10236C000063E064106007900063E0B41516900001
:10237C0089E0FE900062E075F01E84FC7F00EE2C7C
:10238C00F535801C90008BE02535FE900089E02E01
:10239C00FE900062E075F01E84FC7F00EE2CF5359B
:1023AC0022900062E075F00584FF7E008F3690006D
:1023BC0062E075F00584ADF07C008D39753E0575D5
:1023CC005903755AD69000DDE01475F00584FF7E34
:1023DC0000E536BE00039F5005120C5D800BE53600
:1023EC00900462126AD2E0F536E5369008BBF090A4
:1023FC0008BBE0FE9000CCE0C39E50089000CCE0FF
:10240C009008BBF022E56675F00A84FF7E0090050B
:10241C008C120048E0F545E545D394644010E54541
:10242C00C3946475F00F84FF7E008F45800375455F
:10243C00009000AFE02545F54522E56675F00A846D
:10244C00FF7E0090058C120048E0C39469505590B3
:10245C0000F9E0C39403502690088EE0FEA3E0FF41
:10246C007404120039E55E126AA1740F8E048F0594
:10247C00FF126A9190088CECF0A3EDF08024900888
:10248C008EE0FEA3E0FF7404120039E560126AA12D
:10249C00740F8E048F05FF126A9190088CECF0A3D8
:1024AC00EDF0800F90088EE0F8A3E090088CC8F057
:1024BC00A3C8F0A203401A90088EE0FEA3E0FF74BC
:1024CC0003126AA1740112003990088CEEF0A3EF8C
:1024DC00F090088CE0FEA3E0FF900892E0FCA3E0F3
:1024EC00FDEDD39FEC9E400F900892E0F8A3E09096
:1024FC00088CC8F0A3C8F09000A2E0B40262E569B1
:10250C00C3944175F00584FF7E008F36E56975F044
:10251C000584ADF07C008D39753E05755906755AEC
:10252C0014E536C394175005120C5D80069006B363
:10253C00E0F53690088CE0FEA3E0FF740A8E048F61
:10254C0005FF126A91E5368C068D07126AA1740A92
:10255C008E048F05FF126A9190088CECF0A3EDF0BD
:10256C0022E50875F004A4FFAEF09006CF120048E7
:10257C00E09032A1F8282873804C855272804790E5
:10258C0000DFE0855EF0A4FFAEF074081200398F16
:10259C00728033856072802E8566728029856772A1
:1025AC008024856872801F856972801A856A7280A2
:1025BC00158565728010856472800B856B72800640
:0625CC00900028E0F5720A
:1032A10002258402258602258B02259F0225A40280
:1032B10025A90225AE0225B30225B80225BD0225A6
:0732C100C20225C70225CC63
:1025D200E50875F004A4FFAEF09006D0120048E5BD
:1025E2000875F004A4FFAEF0E0FC9006D11200489A
:1025F200ECFEE0FFEEC39F40030226DAE50875F029
:1026020004A4FFAEF09006CF120048E0B40441E506
:102612000875F004A4FFAEF09006D1120048E0C3A2
:102622009572500AE508F50CD3922E1240AFE508D8
:1026320075F004A4FFAEF09006D0120048E0D395E6
:1026420072400AE508F50CC3922E1240AF0226D85A
:10265200E50875F004A4FFAEF09006D0120048E041
:10266200C395725015E50875F004A4FFAEF090060C
:10267200D1120048E0D395725002800AE508F50CA9
:10268200D3922E1240AFE50875F004A4FFAEF0908D
:1026920006D0120048E0D395725015E50875F00493
:1026A200A4FFAEF09006D1120048E0C39572500A22
:1026B200E508F50CC3922E1240AF9006D7E0B401A4
:1026C200099000EBE0D395605002800A7402F50C89
:1026D200C3922E1240AF806AE50875F004A4FFAEE3
:1026E200F09006D0120048E0D395724015E50875C7
:1026F200F004A4FFAEF09006D1120048E0C3957238
:102702004002800AE508F50CC3922E1240AFE5089C
:1027120075F004A4FFAEF09006D0120048E0C39515
:10272200724015E50875F004A4FFAEF09006D112D0
:102732000048E0D39572400AE508F50CD3922E12B8
:1027420040AF22AE2DAF2E74C9BE000CD39F4008FD
:10275200782D126AF402285F752E01752D00AE5194
:10276200AF52E545BE000DD39F40099000C1E0D3B2
:10277200954640028023754600E545C39552F572A1
:102782009000C4E0D395444008E5442572F54480A6
:10279200069000C4E0F5448002054690009DE0D317
:1027A2009560401CE55EC3955F4015AE51AF52E5A2
:1027B20045BE00039F50099000C2E0D395474002F6
:1027C200806E9008BDE0A851B80004955250037580
:1027D20049009008BDE0A851B8000BD395524006BD
:1027E200E5529008BDF0E5497041E552C39545F5C3
:1027F20072E572D3940540037572059000C3E0C37D
:1028020095445007E572C3954440028009E544C3EC
:102812009572F54480069000C3E0F5449000C3E051
:10282200D3954440069000C3E0F54475470080020A
:102832000547E549701690009DE0C39560500DE58F
:10284200452405A851B8000695524002800F900019
:10285200B0E0F54475490174789008BDF022AE2DC0
:10286200AF2E74E9D39F74039E4008782D126AF448
:10287200022A06752E01752D00754432A227402AC0
:102882007544199000B0E075F002A4FFAEF0E54681
:10289200BE0006D39F4002D22705467549037478CD
:1028A2009008BDF07548000229EDAE51AF52E545E2
:1028B2006F4E70030229EDE545BE000DD39F40091E
:1028C2009000C1E0D395464002800F754600E5496D
:1028D200C394035003754419800DE545C39552F521
:1028E20072E5462572F54690009DE0D39560400E54
:1028F2009008BDE0A851B80007D395524002800C61
:1029020005489000B0E0B54803754900E549B403B5
:1029120006A203B3B34002800A0548E548B43C036B
:10292200754902E549B402299008BDE0A851B800F2
:102932000ED395524009E5529008BDF075480090BB
:10294200009DE0C39560500975480074789008BDF9
:10295200F0E549705A90009DE0D39560401CE55E19
:10296200C3955F4015AE51AF52E545BE00039F507F
:10297200099000C2E0D39547400280087547007570
:10298200444B8028E552C39545F572E572D3940510
:10299200400375720590009DE0D395604008E547BD
:1029A2002572F5478006E5472406F547754800E598
:1029B20049701690009DE0C39560500DE5452405D1
:1029C200A851B80006955240028003754901E549B5
:1029D200B4011875441905489000B0E0B548067571
:1029E200490275480074789008BDF0A201B3400313
:1029F200754432E54475F00AA4FFAEF0900894EEF7
:102A0200F0A3EFF022E56E9032C8F8282873900008
:102A120095E07003022C449000CBE0B401028003E5
:102A2200022B4F900060E0655D6009E55245516000
:102A320003022B4C7E017F00E5BE126AA1E5BD2F89
:102A4200FF50010E8E598F5A7410126AA190007DA8
:102A5200E08E048F05FF126A91900898ECF0A3EDC6
:102A6200F0E56A600FE56AC394FE50089000F1E059
:102A72006402600280649000DFE0B40B1F9008984B
:102A8200E0FEA3E0FF74E7126AA1E56A8E048F05F7
:102A9200FF126A91900898ECF0A3EDF09000DFE04D
:102AA200D3940B40089000C7E064046002802B902E
:102AB2000898E0FEA3E0FF90089CE0FCA3E0FDEF95
:102AC200D39DEE9C400D126AEC900898EEF0A3EFB5
:102AD200F08007900898E4F0A3F0900095E0B4022B
:102AE2002790089AE0FEA3E0FF900898E0FCA3E09C
:102AF200FDEF2DFDEE3CFC74018C068D07120039B2
:102B0200900898EEF0A3EFF0900898E0FEA3E0FFA3
:102B120090089AE0FCA3E0FDEDD39FEC9E4004D226
:102B22002B8002B22B900898E0F8A3E090089AC894
:102B3200F0A3C8F09000C7E064016006A22BB3B313
:102B420040028006900899E0F55E022C42D22B7E6C
:102B5200017F00E5BE126AA1E5BD2FFF50010E8E76
:102B6200598F5A7410126AA190007DE08E048F056D
:102B7200FF126A91900898ECF0A3EDF0E56A600FFD
:102B8200E56AC394FE50089000F1E064026002809E
:102B9200649000DFE0B40B1F900898E0FEA3E0FF12
:102BA20074E7126AA1E56A8E048F05FF126A91909A
:102BB2000898ECF0A3EDF09000DFE0D3940B40080E
:102BC2009000C7E064046002802B900898E0FEA3A6
:102BD200E0FF90089CE0FCA3E0FDEFD39DEE9C405B
:102BE2000D126AEC900898EEF0A3EFF080079008BF
:102BF20098E4F0A3F0900095E0B4022790089AE0E0
:102C0200FEA3E0FF900898E0FCA3E0FDEF2DFDEEAF
:102C12003CFC74018C068D07120039900898EEF086
:102C2200A3EFF0900898E0F8A3E090089AC8F0A308
:102C3200C8F09000C7E064016006900899E0F55E74
:102C42008003755E00900091E07006756E01022AA5
:102C52000775BB1802327B900091E07003022DCA07
:102C62007E017F00E5BE126AA1E5BD2FFF50010E75
:102C72008E598F5A9000D7E0B4010F7E0F7FFFACC0
:102C820059AD5A126AEC8E598F5A9000FCE0B40288
:102C920045AE59AF5A900031E0FCA3E0FDEDD39F61
:102CA200EC9E400A900031E559F0A3E55AF0AE5986
:102CB200AF5A900033E0FCA3E0FDEFD39DEE9C40C1
:102CC2000A900033E559F0A3E55AF0AE59AF5A74B1
:102CD200041200398F609000FCE0704CAE59AF5A7C
:102CE200900031E0FCA3E0FDEFD39DEE9C40091281
:102CF2006AEC8E598F5A8006755A00755900AE5982
:102D0200AF5A7410126AA190007AE08E048F05FF08
:102D1200126A918C598D5A74FFBC0009D39D4005EB
:102D2200855A6080037560FE9000C7E0B40102809E
:102D320003022DC8A203B3B3500E90009BE0A8512A
:102D4200B80005D39552500280719000D8E085609A
:102D5200F0A4FFAEF074648E048F05FF126A918CAA
:102D6200598D5AE56A6016E56AC394FE500F9000C9
:102D7200F1E0B402089000DFE0640B60028017AE5D
:102D820059AF5A74E7126AA1E56A8E048F05FF12E1
:102D92006A918C598D5AAE59AF5A900898E0FCA3AB
:102DA200E0FDEDD39FEC9E4005855A5E800BA22B81
:102DB200B34006900899E0F55E800BA22BB3400663
:102DC200900899E0F55E8003756000900094E070D1
:102DD20006756E02022A0775BB1902327B900094B7
:102DE200E07003022E7FE55DD395504003022E7DF5
:102DF20090002FE0FEA3E0FFE564126AE490002F4A
:102E0200EEF0A3EFF07E017F00E5BE126AA1E5BD00
:102E12002FFF50010E8E598F5A900101E0701374EA
:102E22000A126AA174518E048F05FF126A918D6491
:102E32008019AE59AF5A740A126AA18F048E057EA8
:102E4200017F95CDCCCD12698F8F64E564D39464F4
:102E5200400375646490002FE0FEA3E0FFE5642F59
:102E6200FF50010E90002FEEF0A3EFF0900098E0DB
:102E7200048E048F05FF126A918D6480037564329B
:102E82009000E4E07006756E03022A0775BB130218
:102E9200327B9000E4E0604A7E017F00E5BE126A68
:102EA200A1E5BD2FFF50010E8E598F5A74041200F6
:102EB200398F659000E6E08565F0A4FDACF074649E
:102EC200FF126A918D659000E5E08565F0A4FFAE82
:102ED200F074FF8E048F05FF126A91ED900079F075
:102EE2008003756500900092E07006756E04022AF8
:102EF2000775BB1702327B900092E0B40102800397
:102F0200022F8D7E017F00E5BE126AA1E5BD2FFF73
:102F120050010E8E598F5A9008BEE060199008BE7B
:102F2200E01490649C12008CE493FC740193FDED18
:102F3200C39FEC9E400280069008BEE014F0900809
:102F4200BEE0C394B3501DAE59AF5A9008BEE00420
:102F520090649C12008CE493FC740193FDEFC39D7A
:102F6200EE9C400280069008BEE004F09008BEE0AD
:102F7200FE9000B8E08E0088F0A4FFAEF074648E7C
:102F8200048F05FF126A918D6680037566009000BA
:102F920093E07006756E05022A0775BB1602327B36
:102FA200900093E0B4010280030230367E017F007C
:102FB200E5BE126AA1E5BD2FFF50010E8E598F5A50
:102FC2009008BFE060199008BFE0149066061200F6
:102FD2008CE493FC740193FDEDC39FEC9E40028050
:102FE200069008BFE014F09008BFE0C394B3501DF0
:102FF200AE59AF5A9008BFE00490660612008CE406
:1030020093FC740193FDEFC39DEE9C4002800690F9
:1030120008BFE004F09008BFE0FE9000BEE08E0022
:1030220088F0A4FFAEF074648E048F05FF126A91DB
:103032008D67800375670075BB1F02327B7E017F3F
:1030420000E5BE126AA1E5BD2FFF50010E8E598F19
:103052005A7409126AA174E68E048F05FF126A91EE
:103062008D6990009AE07006756E07022A0775BB9B
:103072001502327B90009AE070030231C77E017F15
:1030820000E5BE126AA1E5BD2FFF50010E8E598FD9
:103092005A74041200398F6890009AE0B4011590B6
:1030A20000EEE08568F0A4FFAEF07407120039EF7D
:1030B2009008B9F090009AE0B402159000EEE08515
:1030C20068F0A4FFAEF07407120039EF9008B8F070
:1030D20090009AE0B4030280030231AA9000DBE080
:1030E2007052E568C39419500FD2269000BAE0904E
:1030F20008BCF09008C0E4F0E568D394644004A2F0
:10310200264002802D9008C0E004F09008C0E0FE46
:1031120090012DE0B5060B9008BCE004F09008C0C9
:10312200E4F09008BCE06496600690012DE0700225
:10313200C22680639000BAE070349000EEE08568A9
:10314200F0A4FFAEF074FF8E048F05FF126A91EDBA
:103152009008BCF0AE51AF52741EBE0006D39F4021
:1031620002D226E560D394E54002C2268029E568B2
:10317200C3940A500DAE51AF52741EBE0004D39FC9
:1031820050028002D226E560D394E54002C2269026
:1031920000BAE09008BCF09008BCE0C39405500669
:1031A20074059008BCF0C22C90009AE0B40414E5B7
:1031B20068C394195002D22CE568D394324002C2FB
:1031C2002CC22680037568009000F1E07006756ECF
:1031D20008022A0775BB1402327B9000F1E07003EB
:1031E20002326A7E017F00E5BE126AA1E5BD2FFFB1
:1031F20050010E8E598F5A900116E07025EFD3942C
:1032020021EE940E4005756AFF8015AE59AF5A74CF
:1032120010126AA174E38E048F05FF126A918D6AFF
:103222008027AE59AF5AEFD39449EE940640057504
:103232006AFF8015AE59AF5A7410126AA174658E76
:10324200048F05FF126A918D6AE56A75F00BA4FF7F
:10325200AEF09000DFE08E048F05FF126A919008B5
:103262009CECF0A3EDF08003756A00900095E0609D
:093272000575BB1A800375BB1839
:1032C800022A10022C59022DDF022E94022EF90236
:0B32D8002FA202303F0230760231DCF2
:05327B00056ED2EC22FB
:096AD2002582F5825002058322A1
:0F008C0025E050020583258250020583F582226C
:106A7000EF2F500205832582F582E5833E2EF583B4
:016A800022F3
:106AE400CFC39FFF50011E22C3EF9DFFEE9CFE22E9
:086AF4000806B6000218062294
:0D6AAF00A3E004F07006126AC8E004F022B3
:0E003900048007C3CE13CECF13CFD5E0F6223E
:10698F00BC000FBE0008ED8FF084FFADF022E4FED7
:10699F00FF22BE000DEF60FE54F0606F20E7030290
:1069AF006A45EAC0E0EBC0E078017A0075F001EECD
:1069BF0020E710EF25E0FFEE33FE0AC5F023C5F008
:1069CF0030E7F0EA5407F9096A7A007B00600108A2
:1069DF00C3EC9E40167004ED9F4010ED9FFDEC9EA2
:1069EF00FCE5F0CA4ACA03F5F08005E5F003F5F0BF
:1069FF00C3EE13FEEF13FFD9D77908CACBCAD8D08D
:106A0F00EAFEEBFFD0E0FBD0E0FA22EC8FF084FC43
:106A1F00ED54F045F0C48FF084FEEDC454F045F012
:106A2F00C48FF084FDEEC4FE54F02DFFEE540F3CE6
:106A3F00FEADF07C0022790078008FF0EC7E08200C
:106A4F00E70DC3CD33CD33C933C9C833C8DEF084A6
:106A5F0049F9E5F08FF0BE00E6FD7C00E9FFE8FEA6
:016A6F002204
:0E6AA100F88FF0A4FFE5F0CE88F0A42EFE22C0
:10000300EF8DF0A4F9A8F0EF8CF0A428F8EE8DF0B2
:06001300A428FEE9FF2213
:106A8100600D782B026A8B007830D8FED5E0F822B1
:106A9100EEC0E07E0012698FEFFDEEFCD0E0FE2239
:0C6ABC00EEC0E07E0012698FD0E0FE22E8
:03001B0002001EC2
:0300530002005652
:03009B00020071EF
:03000000026ADBB6
:096ADB0075817475D0000242902F
:0B004800E5822FF582E5833EF5832260
:0A6AC8000582D58202158315822293
:10001E00C0E0C0F0C083C082C0D075D000124234A0
:0B002E00D0D0D082D083D0F0D0E032E0
:10005600C0E0C0F0C083C082C0D075D00012423765
:10006600D0D0D082D083D0F0D0E032C0E0C0F0C093
:1000760083C082C0D075D000124259D0D0D082D071
:0600860083D0F0D0E0324F
:00000001FF
